:020000040800F2
:10000000503D00209D0100088D1B00089D17000831
:10001000891B000881120008D92400080000000094
:1000200000000000000000000000000005010008C2
:100030006D1400080000000049010008B51E00080A
:10004000B7010008B7010008B7010008B7010008B0
:10005000B7010008B7010008B7010008B7010008A0
:10006000B7010008B7010008B7010008B701000890
:10007000B7010008B7010008B7010008B701000880
:10008000B7010008B7010008B7010008B701000870
:10009000B7010008B7010008B7010008B701000860
:1000A000B7010008B7010008B7010008B701000850
:1000B000B7010008B7010008B7010008B701000840
:1000C000B7010008B7010008B7010008B701000830
:1000D000B7010008251F0008412000085D21000825
:1000E000B7010008B7010008B7010008DFF810D019
:1000F00000F0D8FC00480047F9510008AFF3008039
:10010000503D0020224B19680868B0E8F00F80F3DA
:100110000988BFF36F8F4FF0000080F311884EF015
:100120000D0E70470000000006480068006880F36C
:10013000088862B661B6BFF34F8FBFF36F8F00DFE1
:1001400000BF00BF08ED00E0EFF30980BFF36F8F41
:100150000F4B1A6820E9F00F106008B54FF05000FF
:1001600080F31188BFF34F8FBFF36F8F08F000FD4E
:100170004FF0000080F31188BDE808401968086856
:10018000B0E8F00F80F30988BFF36F8F704700BFAE
:100190003C010020EFF305807047000006488047CF
:1001A00006480047FEE7FEE7FEE7FEE7FEE7FEE75C
:1001B000FEE7FEE7FEE7FEE7C51E0008ED000008CB
:1001C00040EA01039B0703D009E008C9121F08C0D9
:1001D000042AFAD203E011F8013B00F8013B521E59
:1001E000F9D27047D2B201E000F8012B491EFBD2D0
:1001F00070470022F6E710B513460A460446194632
:10020000FFF7F0FF204610BD10B5044604E00B7860
:1002100000F8013B03B1491C521EF8D2204610BD24
:10022000421C10F8011B0029FBD1801A704710B541
:10023000002200E0521C835C8C5CA34201D1002BA5
:10024000F8D1D8B2E1B2401A10BD30B50546002051
:10025000034600E05B1C934205D2EC5CC85C201AAC
:1002600001D1002CF6D130BD2DE9F05F93460F4649
:1002700080460446002602F0DBF9D0F80090824662
:1002800014F8015B2DB100F017FA0068405DC0075B
:10029000F6D12B2D02D02D2D1AD0641E0021CAF8C4
:1002A00000105A463946204600F00AFA014627B1A6
:1002B0003868A04201D1C7F80080DAF800000228AF
:1002C00009D0CAF80090700505D54842BDE8F09FF6
:1002D00046F48066E2E70846F8E770B5064602F0A5
:1002E000A7F9046805460A220021304600F037FAD3
:1002F0002C6070BD80EA010210B502F0004340009E
:1003000022D04A001FD0010E01EB1261C0F356004B
:10031000C2F3560240F4000042F40002A0FB0220A7
:1003200000047F39140400D0401C50EA124001D46C
:100330004000491EC2B20C0604EBD010401C40081D
:10034000802A02D003E0002010BD20F00100002927
:1003500000DA0020184310BD30B480EA010202F038
:10036000004530F0004221F0004013D090B1C30DA1
:10037000D40DC2F31601C0F31600E41A41F40001D3
:1003800040F400027D34914201D3641C00E0490036
:10039000002C02DA30BC002070474FF4000000232C
:1003A000914201D3891A034340084FEA4101F7D132
:1003B00051B1914202D14FF0004105E002D24FF01D
:1003C000010101E06FF0010103EBC450284430BC8F
:1003D00000F0FDB92DE9FE4F81EA030404F000446A
:1003E00021F0004100944FF0000B23F0004350EA4D
:1003F00001045ED052EA03045BD0C3F30A54C1F394
:100400000A552C44A4F2F3340194A0FB0254C1F326
:10041000130141F48011C3F3130343F4801301FB70
:10042000024400FB034E840A970A44EA815447EAD7
:100430008357A4FB076802958D0A05FB07854FEAE1
:10044000932C04FB0C542705029D4FEA065847EAFB
:100450001637B5EB08056EEB070C870E920E47EAD0
:10046000811742EA8312A7FB0201B6EB0B0164EB92
:1004700000042B0D43EA0C335E1844EB1C50DA46A3
:100480005146E7FB0201C5F313044FEA0B3343EA7D
:1004900014534FEA0432019C43EA0603A4F10C040E
:1004A0000294009CCDE900B400F0D7F903B0BDE898
:1004B000F08F00200146F9E72DE9F04D81EA0304B1
:1004C00004F0004B21F0004514464FF0000A23F0E1
:1004D000004150EA050220D054EA01021DD0C5F3C4
:1004E0000A570246C5F31303C1F31300C1F30A56BA
:1004F00040F4801543F48013A7EB0608101BD64682
:1005000008F2FD3873EB050002D308F1010801E0A1
:1005100092185B41B8F1000F03DA00200146BDE8F4
:10052000F08D00204FF48011064684460EE0171B24
:1005300073EB050705D3121B63EB050306434CEA77
:10054000010C49084FEA300092185B4150EA01075C
:10055000EDD152EA030012D082EA040083EA0501D9
:10056000084305D0101BAB4106D20122002306E050
:1005700000224FF0004302E06FF0010253101AEB2B
:1005800006004CEB085110EB0A0041EB0B01BDE8F3
:10059000F04D00F053B9C10F80EAE0700844CA077B
:1005A0009623002100F01CB996230022114600F08A
:1005B00017B9C1F30A5210B5C1F3130140F2FF336A
:1005C00041F480119A4201DA002010BD40F2334319
:1005D0009A42A2F2334203DC524200F05DF810BDB1
:1005E000904010BD00F0004230F000400AD0C10D34
:1005F00001F56071C0F3160042EA0151C2084007DC
:100600001143704700200146704730B50B46014644
:1006100000202022012409E021FA02F59D4205D3A1
:1006200003FA02F5491B04FA02F52844151EA2F14B
:100630000102F1DC30BD2DE9F05F05460020924655
:100640009B4688460646814640241BE02846414694
:100650004746224600F020F853465A46C01A9141B8
:1006600010D311461846224600F02EFA2D1A67EBD9
:1006700001084F4622460120002100F025FA17EB21
:1006800000094E41201EA4F10104DFDC484631463A
:100690002A464346BDE8F09F202A04DB203A21FA8F
:1006A00002F00021704721FA02F3D040C2F120028B
:1006B000914008431946704700487047F0A1000870
:1006C0002DE9F05F82460078002715468B460AF137
:1006D0000104B946302801D09DB113E014F8010B94
:1006E0000127782803D0582801D045B10AE00DB180
:1006F000102D07D10027102514F8010B02E0082562
:1007000000E00A250026B0460EE005FB080005FBC8
:1007100006F1012701EB10461FFA80F8B6F5803F7D
:1007200000D3B94614F8010B294600F0EEF9002871
:10073000EBDABBF1000F05D00FB1641E00E05446A8
:10074000CBF80040B9F1000F06D001F071FF022193
:100750000160C81EBDE8F09F48EA0640FAE72DE9AF
:10076000F04791460F4680460446002614F8015B88
:100770002DB1FFF7A1FF0068405DC007F6D12B2D1A
:1007800002D02D2D18D0641E4A4639462046FFF768
:1007900097FF27B13968A14201D1C7F800807105E0
:1007A0004FF002040BD54042002803DD01F040FF6A
:1007B0000460A007BDE8F08746F48066E4E70028FF
:1007C000F8DA01F035FF04606FF00040F2E700292D
:1007D000A8BF7047401C490008BF20F001007047C7
:1007E00010B4B0FA80FC00FA0CF050EA010404BF27
:1007F00010BC704749B1CCF1200421FA04F411FA7D
:100800000CF118BF012121430843A3EB0C01CB1DC0
:100810004FEA00614FEA102042BF002010BC704731
:1008200000EBC35010440029A4BF10BC7047401C0B
:10083000490008BF20F0010010BC704710B5141E1D
:1008400073F1000408DA401C41F1000192185B4189
:100850001A4301D120F0010010BD2DE9F04D924660
:100860009B4611B1B1FA81F202E0B0FA80F2203277
:10087000904600F029F904460F4640EA0A0041EA92
:100880000B0153465A46084313D0114653EA010060
:1008900019D0C8F140025046FFF7FEFE05460E464D
:1008A00050465946424600F00FF9084305D0012052
:1008B00004E020463946BDE8F08D0020054346EAB5
:1008C000E0762C4337430A986305E40AA0EB08005E
:1008D0000022FD0A44EA47540A3002D500200146AE
:1008E000E9E7010510196941DDE908450019694189
:1008F000BDE8F04DA2E72DE9FE4F804681EA0300F6
:10090000C00F0C46009021F0004123F00045B8EBE9
:100910000200A94105D24046214690461C460B469E
:10092000024623F00040104347D0270DC7F30A00CA
:10093000C3F30A510290401A019040286BDAC3F3C6
:10094000130040F4801B0098924620B10023D2EBA4
:10095000030A63EB0B0B01985946C0F14002504665
:1009600000F0B2F806460D4650465946019A00F08E
:10097000BAF810EB08006141002487EA115284EABA
:10098000E7731A4340D0009A62B3019A012A4FEAF2
:10099000075215DC001B61EB02014FF0004202EA36
:1009A0000752CDE90042001C41F5801132462B462A
:1009B000FFF753FF03B0BDE8F08F40462146F9E74B
:1009C000001B61EB0201001C41F5801300185B4124
:1009D0002018A2F5001747EB030140EAD570B619BD
:1009E0006D4111E06D084FEA360645EAC0754FEAE1
:1009F0000752001B61EB0201001C41F58011490800
:100A00004FEA30000019514132462B4603B0BDE891
:100A1000F04FFFF713BF0098012240000023D0EBF6
:100A2000020263EBE073009821464FEAE074B8EBF2
:100A3000000061EB0401E9E783F000435BE781F02C
:100A4000004158E7C1F30A52C1F3130140F2FF33EA
:100A500041F480119A4202DA00200146704740F2C8
:100A600033439A42A2F2334202DC5242FFF714BEF1
:100A700000F02AB830B5041E71F1000404DB4FF019
:100A80000044404264EB0101141E73F1000405DBD5
:100A90001C464FF00043524263EB0403994208BFE7
:100AA000904230BD064C074D06E0E06840F001037F
:100AB00094E8070098471034AC42F6D3FFF71AFBCE
:100AC00044A6000864A60008202A04DB203A00FAA5
:100AD00002F1002070479140C2F1200320FA03F395
:100AE000194390407047202A06DBCB17203A41FA81
:100AF00002F043EAE07306E041FA02F3D040C2F1AB
:100B0000200291400843194670473A2800D23038F5
:100B100020F02002412A01D3A2F13700884201D3FC
:100B20004FF0FF30704770B58C1810F8015B15F06E
:100B3000070301D110F8013B2A1106D110F8012B4F
:100B400003E010F8016B01F8016B5B1EF9D12B0774
:100B500005D40023521E0DD401F8013BFAE710F82A
:100B6000013BCB1A921C03E013F8015B01F8015B17
:100B7000521EF9D5A142D8D3002070BD00B591B066
:100B80000121042001F084F82020ADF8400000206D
:100B90008DF8430010A9394800F00FFD01210846E7
:100BA00001F056F80121480201F072F8344800F0D3
:100BB00099FB3448009034480190002002900120B5
:100BC0000390002004908020059040000690800053
:100BD0000790202008900002099000200A906946A2
:100BE000274800F025FC0121254800F06FFB00207C
:100BF0000B9001208DF830008DF831004FF460200B
:100C00000D9000200E9001208DF83C000BA91D488E
:100C10004C3800F065F84FF4404001F00DF8052322
:100C20000122194617484C3800F082F80121154876
:100C30004C3800F036F8012112484C3800F026F804
:100C400010484C3800F0D0F800BF0E484C3800F087
:100C50003DF80028F9D10B484C3800F0D5F800BF1A
:100C600008484C3800F028F80028F9D1012105483F
:100C70004C3800F0BEF811B000BD00000008014083
:100C8000080002404C2401405003002021B182683A
:100C900042F00102826003E0826822F00102826079
:100CA000704721B1826842F48072826003E08268FA
:100CB00022F4807282607047014600208A6802F048
:100CC00004020AB1012000E0002070470146002024
:100CD0008A6802F008020AB1012000E00020704793
:100CE00030B502460020002350680F4C20400D799B
:100CF0000C6844EA05242043506090680B4C204067
:100D0000D1E902542C434D7944EA450420439060D4
:100D1000D06A20F470000C7C641EE4B2234340EAE5
:100D20000350D06230BD0000FFFEF0FFFDF7F1FF81
:100D3000F0B504460D4600200021092D11DDE068C4
:100D4000A5F10A0606EB4607072606FA07F18843CF
:100D5000A5F10A0606EB460603FA06F10843E06031
:100D60000CE0206905EB4507072606FA07F18843E2
:100D700005EB450603FA06F108432061072A0FDA5E
:100D8000606B561E06EB86071F2606FA07F188439E
:100D9000561E06EB860605FA06F10843606322E05C
:100DA0000D2A0FDA206BD61F06EB86071F2606FAE0
:100DB00007F18843D61F06EB860605FA06F10843BD
:100DC000206310E0E06AA2F10D0606EB86071F26FD
:100DD00006FA07F18843A2F10D0606EB860605FA2E
:100DE00006F10843E062F0BD816841F008018160CE
:100DF000704721B1826842F4A002826003E08268F9
:100E000022F4A00282607047816841F00401816091
:100E10007047000008B50121082000F039FF4FF4A9
:100E20008070ADF8000010208DF8030003208DF8CD
:100E300002006946014800F0C0FB08BD000C0140FB
:100E40007CB5012407F014FB3148022100230A027B
:100E5000CDE900102FA1324808F076FB0446012CA2
:100E600002D030A001F094FB36480221002340223A
:100E7000CDE9001034A1374808F066FB0446012C88
:100E800002D035A001F084FB3B480068022100231A
:100E90000A02CDE9001039A13B4808F055FB044691
:100EA000012C02D039A001F073FB404800680221F8
:100EB00000234022CDE900103DA1404808F044FB4A
:100EC0000446012C02D03EA001F062FB44480123FD
:100ED0001A464FF47A71009042A008F091FD4449FF
:100EE00008600846006858B108F06EFB054600200F
:100EF00003462A46012100903D48006808F0D4FDD1
:100F00003C48006807F060FC07F0F4FA7CBD000084
:100F1000040000204D61696E5F5461736B00000036
:100F2000D1180008E5889BE5BBBA4D61696E5F5436
:100F300061736BE4BBBBE58AA1E5A4B1E8B4A5216C
:100F40000D0A0000080000204B65795F5461736B47
:100F500000000000E5170008E5889BE5BBBA4B657B
:100F6000795F5461736BE4BBBBE58AA1E5A4B1E88A
:100F7000B4A5210D0A0000000C00002057646F6723
:100F80005F5461736B00000047250008E5889BE50E
:100F9000BBBA57646F675F5461736BE4BBBBE58A90
:100FA000A1E5A4B1E8B4A5210D0A000010000020BD
:100FB0004261745F5461736B0000000051120008BD
:100FC000E5889BE5BBBA4261745F5461736BE4BB17
:100FD000BBE58AA1E5A4B1E8B4A5210D0A00000093
:100FE000817E000874696D655F6C6F636B00000043
:100FF000140000200000002008B501210C2000F0A2
:1010000047FE1020ADF8000048208DF80300694627
:10101000064800F0D2FA0420ADF8000048208DF810
:1010200003006946024800F0C8FA08BD0008014004
:10103000000C014070B51B480068401C194908604D
:101040000421194800F08CFB05461021174800F0D8
:1010500087FB0446C4B9012D16D1124800681E282A
:101060001EDB11480C300168012088430E490C3109
:10107000096801F0010140EA01400B4910310860A4
:101080000020084908600BE0012C05D125B9012199
:10109000054800F06EFB03E00121034800F06BFB04
:1010A000002070BD20000020000C0140000801401D
:1010B00008B50121042000F0EBFD0220ADF800008E
:1010C00010208DF8030003208DF8020069460448C3
:1010D00000F073FA0221024800F04DFB08BD000049
:1010E0000008014010B54FF4407000F089FD02F097
:1010F00065FC2D4908688047FFF78CFE2B48016886
:101100004FF4E1308847294881684FF416508847EA
:10111000264841684FF4165088472448052224A1E8
:10112000C3682548984725490868804724490868C6
:10113000804704F0A5FF0121017004F0A1FF002108
:10114000417004F09DFF0021017204F099FF00211D
:10115000C1714FF480711B4800F00BFB4FF42F70EE
:1011600002F04EFC4FF42F7002F04AFCFFF7A0FF94
:101170000D4841680120884700F04CFD02F0E8FC72
:1011800018B905F065F805F04BF803E000F07AF8BF
:1011900000B900E0FAE700BF01F0C4F906F09EFFD5
:1011A00007F038F810BD00002C000020440000209B
:1011B0007374617274000000004800401800002041
:1011C00024000020000C014038B5044605F0C0FDA5
:1011D0000546032C16DB142C14DC0020009022465C
:1011E0000AA1684601F0FEF9694609A003F048F833
:1011F00003F044F804F044FF8472214606A001F095
:10120000C7F902E00AA001F0C3F938BD2564000067
:101210006B65795F73000000E8AEBEE7BDAEE6889F
:1012200090E58A9F2025642073200D0A00000000AD
:10123000E8AEBEE7BDAEE5A4B1E8B4A52CE8AFB713
:10124000E6A380E69FA5E58F82E695B0200D0A0013
:1012500003E04FF47A7007F079FAFAE7064801687C
:10126000012088430449096801F0010140EA014076
:1012700002490860704700000C0C01401008014052
:1012800000BFFEE710B501210F4800F069FA48B928
:101290001E2002F0B5FB01210B4800F061FA88B96D
:1012A000002010BD0121084800F05AFA012809D198
:1012B0001E2002F0A5FB0121034800F051FA01288D
:1012C00000D1EEE70020ECE70008014021B1026800
:1012D00042F00102026004E002684FF6FE731A4019
:1012E0000260704701684FF6FE72114001600021F4
:1012F000016041608160C1604B49884208D14A4920
:101300000839496841F00F01474A083A51608AE0BC
:1013100045491431884208D143490839496841F0A8
:10132000F001414A083A51607DE03F492831884246
:1013300008D13D490839496841F470613A4A083A90
:10134000516070E038493C31884208D1364908394B
:10135000496841F47041344A083A516063E03249C7
:101360005031884208D130490839496841F4702128
:101370002D4A083A516056E02B496431884208D121
:1013800029490839496841F47001274A083A5160EF
:1013900049E025497831884208D12349083949680C
:1013A00041F07061204A083A51603CE01F49884290
:1013B00006D1011F096841F00F01021F116032E0E0
:1013C0001A491431884208D11849091F096841F0A7
:1013D000F001164A121F116025E014492831884295
:1013E00008D11249091F096841F470610F4A121FA0
:1013F000116018E00D493C31884208D10B49091FA2
:10140000096841F47041094A121F11600BE0074955
:101410005031884207D10549091F096841F47021FC
:10142000024A121F1160704708000240080402407F
:1014300010B50022026847F6F0739A430C6A8B6875
:1014400023430C6923434C6923438C692343CC69B0
:1014500023434C6A23438C6A23431A430260CB68BC
:1014600043600B6883604B68C36010BD7047000029
:101470000149C860704700000020024030B50446B2
:1014800004254FF4302000F085F80546042D17D1CF
:101490000C48006940F002000A49086108464461AE
:1014A000006940F0400008614FF4302000F072F80D
:1014B00005460448006941F6FD710840014908618C
:1014C000284630BD0020024004200B49C96801F0C5
:1014D000010109B101200EE00749C96801F00401CA
:1014E00009B1022007E00449C96801F0100109B1FF
:1014F000032000E0042070470020024003480069F8
:1015000040F080000149086170470000002002405F
:1015100078B506460C46042500200090E80200F04D
:1015200039F80546042D24D11348006940F0010024
:10153000114908613480E80200F02CF80546042DBA
:1015400010D1B01C0090200C00990880E80200F037
:1015500021F805460848006941F6FE710840064931
:10156000086106E00448006941F6FE71084002493E
:101570000861284678BD0000002002400248034967
:1015800048600348486070472301674500200240D7
:10159000AB89EFCD00B502460423FFF795FF034664
:1015A00003E0FFF791FF0346521E012B01D1002AF1
:1015B000F7D102B90523184600BD2DE9F0410246D6
:1015C00000250026002000230024002791F803C0F6
:1015D0000CF00F0591F803C00CF0100CBCF1000FDB
:1015E00003D091F802C04CEA050591F800C0BCF1A7
:1015F000000F31D0146800202BE04FF0010C0CFAE2
:1016000000F3B1F800C00CEA03069E4220D183002B
:101610004FF00F0C0CFA03F7BC4305FA03FC4CEA3D
:10162000040491F803C0BCF1280F06D14FF0010C5F
:101630000CFA00FCC2F814C00AE091F803C0BCF137
:10164000480F05D14FF0010C0CFA00FCC2F810C095
:10165000401C0828D1D31460B1F800C0BCF1FF0FC2
:1016600034DD546800202EE000F1080C4FF0010832
:1016700008FA0CF3B1F800C00CEA03069E4221D12F
:1016800083004FF00F0C0CFA03F7BC4305FA03FC80
:101690004CEA040491F803C0BCF1280F05D100F115
:1016A000080C08FA0CF8C2F8148091F803C0BCF1D9
:1016B000480F07D100F1080C4FF0010808FA0CF8A8
:1016C000C2F81080401C0828CED35460BDE8F081D9
:1016D000F0B50A46002300240021002500F0004652
:1016E000B6F1004F02D11D4EF16901E01B4E716849
:1016F000C0F3034583B200F44016B6F5401F08D18D
:1017000021F07061154E766826F07066134F7E608A
:1017100012E000F48016B6F5801F06D1032606FA03
:1017200005F4A14341F0706106E0460D360103FA6D
:1017300006F6B14341F0706122B1460D360103FA5D
:1017400006F6314300F00046B6F1004F02D1034ED9
:10175000F16101E0014E7160F0BD00000000014048
:101760000246002093680B400BB1012000E00020EE
:101770007047416170470161704700000648016889
:10178000802088430449096801F0800140EA014053
:101790000149091D086070470C08014000BFFEE7C1
:1017A0004CF6CC4001490860704700000030004012
:1017B0004AF6AA2001490860704700000030004046
:1017C00001494860704700000030004001498860CE
:1017D0007047000000300040014908607047000079
:1017E0000030004004E003F031F80A2006F0AEFFBC
:1017F000F9E7000008B501210C2000F049FA0120AA
:10180000ADF8000010208DF8030003208DF80200D1
:1018100069460C48FFF7D1FEC020ADF8000010204B
:101820008DF8030003208DF8020069460648FFF793
:10183000C4FEC0210448FFF79EFF01210148FFF7C5
:101840009AFF08BD000C01400008014010B5044695
:10185000062C36D2DFE804F003151A101F284021A9
:101860001948FFF788FF80211748FFF784FF0121FF
:101870001648FFF780FF25E001211448FFF779FFA4
:1018800020E080211048FFF774FF1BE040210E4844
:10189000FFF76FFF16E040210B48FFF76AFF80213A
:1018A0000948FFF766FF0DE040210748FFF761FF99
:1018B00080210548FFF75DFF01210448FFF759FF2C
:1018C00000E000BF00BF10BD00080140000C014057
:1018D0001CB506E104F0D4FB0078012873D104F0B4
:1018E000CFFB40780028F9D17E4841680020884726
:1018F0007D48416800208847AA2804DD794841686E
:101900000120884703E0774841680420884704F0B5
:10191000B7FBC07901280FD1724841680020884781
:10192000704988687149322307220C687049A047C2
:1019300004F0A6FB0021C17104F0A2FB007A01288B
:1019400054D104F09DFB0021017204F099FB8078D2
:1019500020B904F095FBC078012804D004F090FB76
:101960008078002830D004F08BFB447904F088FBA9
:10197000057904F085FBC67804F082FB877833464E
:101980003A465CA16A48CDE9005400F02BFE554868
:10199000416800208847674836226549C368664821
:1019A00098475049886851494FF4C87304220C681D
:1019B0004F49A0474B4841680020884704F060FB2E
:1019C000002101700DE011E0464841680020884781
:1019D0004449C86845494FF4C87304220C68444917
:1019E000A04704F04DFB0021C0F8021004F048FBB2
:1019F000007801286BD104F043FB4078012866D1C0
:101A000038484168052088474C48007855285ED101
:101A10004A484078AA285AD104F032FB002181714B
:101A2000464880780D2824D2DFE800F02307080913
:101A30000A0B0C0D0E0F1011120000BF00BF00BFEB
:101A400000BF00BF00BF00BF00BF00BF00BF00BF9E
:101A50003A488078401E3A4901EB0014D4E902016B
:101A6000CDE9000137A13248D4E9002300F0BAFDE6
:101A700000E000BF00BF2F4836222D49C3682E4822
:101A8000984714212D48FEF7B4FB16484168002002
:101A900088471449886815494FF4C87304220C68B4
:101AA0001349A0470F4841680020884704F0E8FA2E
:101AB0000021017004F0E4FA002141704FF4FA6053
:101AC00006F044FE4FF480712D48FFF752FE04F0FB
:101AD000D7FA007810B92B4948688047142006F0DF
:101AE00035FEF7E62C0000202400002078000020BE
:101AF0004D87000841542B4C5253454E443D3835D8
:101B00002C312C33332C227B2245223A222564228D
:101B10002C2254223A222564222C2252223A2225B7
:101B200064222C2243223A222564227D220D0A00BF
:101B30005002002044000020004800409C08002083
:101B40007C00002041542B4C5253454E443D3835C7
:101B50002C312C33332C227B2245223A222573222E
:101B60002C2254223A222573222C2252223A222558
:101B700073222C2243223A222573227D220D0A0051
:101B8000000C01401800002000BFFEE77047000075
:101B900070B5002100230F22C47804B3154C2468CB
:101BA00004F4E064C4F5E064210AC1F10403CA400E
:101BB000447804FA03F184781440214309010E4C5F
:101BC0000678A155047804F01F050124AC4005787F
:101BD0006D11AD0005F1E025C5F8004109E004787C
:101BE00004F01F050124AC40044D0678761145F839
:101BF000264070BD0CED00E000E400E080E100E074
:101C000002490143024A1160704700000000FA05D2
:101C10000CED00E008B50121042000F039F80120A6
:101C2000ADF8000028208DF8030069460148FFF751
:101C3000C4FC08BD0008014001460020034A50686A
:101C400020F44040084350607047000000100240FC
:101C500029B1064A52690243044B5A6104E0034A1F
:101C600052698243014B5A617047000000100240E4
:101C700029B1064AD2690243044BDA6104E0034AFF
:101C8000D2698243014BDA617047000000100240C4
:101C900029B1064A92690243044B9A6104E0034A5F
:101CA00092698243014B9A61704700000010024024
:101CB00030B500210022002400232D4D6D6805F071
:101CC0000C0121B1042905D0082923D105E0294DB3
:101CD000056022E0274D05601FE0254D6D6805F485
:101CE0007012234D6D6805F48034022505EB924295
:101CF0001CB9214D554305600BE01D4D6D6805F481
:101D000000351DB11C4D5543056002E0194D55438A
:101D1000056002E0174D056000BF00BF144D6D68FF
:101D200005F0F0010909154D6B5C0568DD40456063
:101D30000F4D6D6805F4E061090A104D6B5C456854
:101D4000DD4085600A4D6D6805F46051C90A0B4D90
:101D50006B5C4568DD40C560054D6D6805F440412C
:101D6000890B074D6B5CC568B5FBF3F5056130BDAC
:101D70000010024000127A0000093D00B00100206E
:101D8000C0010020064801684020884304490968D2
:101D900001F0400140EA01400149091D0860704717
:101DA0000C08014010B500F001F810BD0CB5002082
:101DB000019000903348006840F480303149086059
:101DC00000BF3048006800F4003000900198401CCB
:101DD0000190009818B90198B0F5A06FF1D1294889
:101DE000006800F4003010B10120009001E00020F4
:101DF00000900098012843D12348006840F010006B
:101E0000214908600846006820F003000860084681
:101E1000006840F0020008601A48406819494860AC
:101E20000846406848600846406840F48060486062
:101E30000846406820F47C1048600846406840F43A
:101E4000E81048600846006840F08070086000BFF5
:101E50000C48006800F000700028F9D0094840687C
:101E600020F00300074948600846406840F002003F
:101E7000486000BF0348406800F00C000828F9D112
:101E80000CBD00000010024000200240042808D1D0
:101E90004FF0E021096941F004014FF0E0221161A7
:101EA00007E04FF0E021096921F004014FF0E02242
:101EB0001161704710B507F077FB012801D006F0DB
:101EC000E7FF10BD10B51348006840F0010011494C
:101ED000086008464068104908400E4948600846B6
:101EE00000680E4908400B4908600846006820F465
:101EF000802008600846406820F4FE0048604FF4E7
:101F00001F008860FFF74EFF4FF000600449086033
:101F100010BD0000001002400000FFF8FFFFF6FEB9
:101F200008ED00E010B540F22551124800F0DAF952
:101F300088B140F225510F4800F0ACF90D4800F08F
:101F40008DFA0D490D4A128888540C480088401CAF
:101F50000A4908800CE01021064800F0B6F938B1B3
:101F6000044800880348001D0088012004490870C7
:101F700010BD000000380140B40400205A000020C9
:101F80005800002010B586B0044601210420FFF758
:101F90007FFE01218803FFF77BFE4FF40070ADF850
:101FA000140018208DF8170003208DF8160005A9DD
:101FB0002148FFF702FB4FF48060ADF814000420C5
:101FC0008DF8170005A91C48FFF7F7FA01940020C7
:101FD000ADF80800ADF80A00ADF80C00ADF810003F
:101FE0000C20ADF80E0001A9144800F0CBF9012136
:101FF000124800F05EF9012240F225510F4800F02E
:102000009BF9012240F224410C4800F095F94FF46D
:102010004070FFF7F5FD25208DF8000001208DF8B8
:10202000030004208DF8010000208DF802006846AE
:10203000FFF7AEFD06B010BD0008014000380140BA
:1020400010B540F22551134800F04CF988B140F228
:102050002551104800F01EF90E4800F0FFF90E4916
:102060000E4A128888540D480088401C0B4908808D
:102070000FE01021074800F028F950B1054800880A
:102080000448001D008800200449088001200449FC
:10209000087010BD004400409C0800205E00002035
:1020A0005C00002010B586B0044601210420FFF733
:1020B000EFFD01214804FFF7DBFD0420ADF814001B
:1020C00018208DF8170003208DF8160005A9214867
:1020D000FFF773FA0820ADF8140004208DF81700FC
:1020E00005A91C48FFF769FA01940020ADF8080023
:1020F000ADF80A00ADF80C00ADF810000C20ADF8FA
:102100000E0001A9144800F03DF90121124800F029
:10211000D0F8012240F225510F4800F00DF90122BC
:1021200040F224410C4800F007F94FF44070FFF7EB
:1021300067FD26208DF8000001208DF803000020A7
:102140008DF801008DF802006846FFF721FD06B00A
:1021500010BD0000000801400044004010B540F2EE
:102160002551184800F0BEF888B140F225511548B5
:1021700000F090F8134800F071F91349134A1288DF
:10218000885412480088401C1049088018E010212B
:102190000C4800F09AF898B10A4800880948001DD8
:1021A0000088002009490880074909A000F0F0F9DB
:1021B0004FF4C8710448FEF71CF801200549087067
:1021C00010BD000000480040B00800206200002060
:1021D000257300006000002010B586B00446012180
:1021E0000820FFF755FD01218804FFF741FD4FF45A
:1021F0008060ADF8140018208DF8170003208DF8CA
:10220000160005A92148FFF7D8F94FF40060ADF892
:10221000140004208DF8170005A91C48FFF7CDF91C
:1022200001940020ADF80800ADF80A00ADF80C00EC
:10223000ADF810000C20ADF80E0001A9144800F014
:10224000A1F80121124800F034F8012240F2255192
:102250000F4800F071F8012240F224410C4800F0D0
:102260006BF84FF44070FFF7CBFC27208DF800008F
:1022700001208DF8030003208DF8010000208DF867
:1022800002006846FFF784FC06B010BD000C014058
:102290000048004010B50022002340F66A14A14215
:1022A00000D100BF0A1201249440A3B2DC43048091
:1022B00010BD21B1828942F40052828104E08289FA
:1022C0004DF6FF731A408281704702460020B1F537
:1022D000007F00D100BF13880B400BB1012000E04C
:1022E0000020704770B5024600240023002500201E
:1022F00040F66A16B14200D100BFC1F3421501F0A9
:102300001F03012606FA03F3012D02D196893340FB
:1023100006E0022D02D1168A334001E0968A33404E
:102320000C12012606FA04F41688344013B10CB1DD
:10233000012000E0002070BDF0B503460024002617
:102340000025002040F66A17B94200D100BF1846A8
:10235000C1F3421401F01F06012707FA06F5012C0C
:1023600001D10C3004E0022C01D1103000E0143017
:102370001AB107682F43076002E00768AF430760A0
:10238000F0BD00002DE9F04786B005460E4600245A
:10239000A24600BFA1460027B08900B100BF2F466A
:1023A0002C8A4CF6FF700440F08804432C82AC89E0
:1023B0004EF6F3100440B088318908437189084310
:1023C0000443AC81AC8A4FF6FF400440B08904431B
:1023D000AC8201A8FFF76CFC1F48874202D1DDF8F0
:1023E00010A001E0DDF80CA0A88900F4004040B185
:1023F0000AEBCA0000EB0A1031684900B0FBF1F8A3
:1024000007E00AEBCA0000EB0A1031688900B0FB54
:10241000F1F86420B8FBF0F004012009642101FB0D
:102420001089A88900F4004040B1322000EBC900B7
:10243000B0FBF1F000F00700044308E0322000EBAD
:1024400009106421B0FBF1F000F00F0004432C816F
:1024500006B0BDE8F08700000038014001468888DA
:10246000C0F308007047C1F30802828070472DE96D
:10247000F04107460C46154600260DE014F8011BF6
:102480003846FFF7F0FF00BF40213846FFF71DFF39
:102490000028F9D0701C86B2AE42EFDBBDE8F081B7
:1024A00070B506460C46002500BF615D3046FFF75B
:1024B000DAFF00BF80213046FFF707FF0028F9D080
:1024C0006D1C605D0028F0D100BF40213046FFF751
:1024D000FCFE0028F9D070BD00BFFEE770B50446D1
:1024E0000D4629462046FFF7BEFF00BF802120464B
:1024F000FFF7EBFE0028F9D070BD70B506460C461C
:10250000002500BF615D3046FFF7E8FF6D1C605D90
:102510000028F7D100BF40213046FFF7D6FE002843
:10252000F9D070BD10B545F25550FFF755F90220AE
:10253000FFF746F940F6FF70FFF748F9FFF738F963
:10254000FFF72EF910BD04E0FFF732F91E2006F068
:10255000FDF8F9E70D480168402088430B490968F8
:1025600001F0400140EA01400849091D0860081FC8
:102570000168802088430549096801F0800140EA2C
:1025800001400249091D0860704700000C08014025
:102590000FB4054B10B503A9044A029800F01EF9C8
:1025A00010BC5DF814FB000035490008480200200B
:1025B0000FB47CB50C0009AD01D0611E00E0002114
:1025C000CDE90001064B6A462946089800F006F955
:1025D000002C02D0009A002111707CBC5DF814FB25
:1025E000E32E00080FB4084B10B504A902AA039803
:1025F00000F0F4F8044602A9002000F07DFC20461B
:1026000010BC5DF814FB0000F92E000837B5144625
:102610000846064B6A46214600F0E0F80446694643
:10262000002000F069FC20463EBD0000F92E0008A5
:10263000004870474C02002002E008C8121F08C181
:10264000002AFAD170477047002001E001C1121F33
:10265000002AFBD1704700002DE9FF5F82B0002106
:10266000DDE90430020DDDF840B0034318D044F634
:102670001050A2F2FF3242431514119801281FD0C6
:10268000A5EB0B00401C5FEA000A4FF000064E4F1E
:10269000DFF83891B046504615D5CAF1000413E072
:1026A000119801244AA3012801D16FEA0B01029875
:1026B000119AC0E90031C0E9024206B0BDE8F09FBE
:1026C000CBF10000DFE704460021404A491842EB05
:1026D0000450CDE9001012E0E00707D032463B4637
:1026E00040464946FDF776FE8046894632463B46DF
:1026F00010461946FDF76EFE06460F466410002C84
:10270000EAD1DDE90401DDE90023BAF1000F06DAC0
:10271000FDF760FE42464B46FDF75CFE05E0FDF727
:10272000CBFE42464B46FDF7C7FE04460E4600224E
:10273000284BFEF79FF903D84FF0FF30014607E022
:102740000022254B20463146FEF7D5F8FEF77AF9F0
:10275000102409E0002C0ADB0A220023FDF76BFF9E
:10276000039B30321A55641E50EA0102F2D1641CF8
:10277000039AC4F111031444119A012A03D00122CF
:1027800008430DD10AE0084304D000204FF0110B9C
:10279000119072E7A3EB0B056D1E0DE05B4504DDA8
:1027A0004FF0000205F1010504E003DA4FF00002EA
:1027B000A5F10105002AECD002981199C0E9023177
:1027C000C0E9004579E70000000014400000F03F38
:1027D000300000000000F0430000E03F2DE9FF4F13
:1027E00095B09A46884606460025EEE1252877D121
:1027F00000242746F94A0121039400E0044316F817
:10280000013F203B01FA03F01042F7D130782A282B
:1028100011D06FF02F033078A0F13002092A16D8BA
:10282000039A44F0020402EB820203EB42021044DA
:10283000761C0390EFE758F8042B0392002A03DA82
:10284000504244F40054039044F00204761C307863
:102850002E2816D116F8010F44F004042A280DD0B2
:102860006FF02F023078A0F13003092B09D807EB65
:10287000870302EB4303C718761CF3E758F8047B81
:10288000761C30786C280FD006DC4C2817D06828CE
:102890000DD06A2814D104E0742810D07A280FD102
:1028A0000DE044F400140AE044F4801401E044F420
:1028B00040147278824202D104F58014761C761C92
:1028C000307866280BD013DC582877D009DC002834
:1028D00075D04528F6D04628F4D047281AD193E180
:1028E00018E0632835D0642879D0652812D18BE1AF
:1028F000702873D008DC6728F1D069286FD06E2863
:102900000DD06F2806D1ACE073282CD0752874D078
:10291000782853D05246179990476D1C54E1C4F360
:102920000250022809D003280DD0D8F8001004283E
:102930000DD00D6008F1040846E1D8F80010EA1740
:10294000C1E90052F6E7D8F800100D80F2E70D70EB
:10295000F0E718F8041B8DF8001000208DF8010036
:10296000EB46012003E058F804BB4FF0FF3061074D
:102970004FF0000102D40DE009F101018946B9428E
:102980000FDA8145F8DB1BF809100029F4D108E0C3
:1029900009F1010189468142FADB1BF8091000297F
:1029A000F6D103985346A0EB090721463846179AFB
:1029B00000F080FA284400EB090507E044E008E154
:1029C0000DE01BF8010B524617999047B9F1010928
:1029D000F7D2534621463846179AF2E039E00A21E9
:1029E000C4F302524FF0000B0091022A06D058F8AF
:1029F000040BC117032A09D00AE023E008F10700FD
:102A000020F00702F2E80201904605E000B2C1178B
:102A1000042A01D140B2C117002906DA0A46002172
:102A2000404261EB02012D2202E0220504D52B2257
:102A30008DF80420012203E0E20701D02022F7E70D
:102A4000914657E00A2100E010214FF0000B009161
:102A50000BE010214FF0000B44F004040827009114
:102A600003E008204FF0000B0090C4F30252022A4A
:102A700005D058F8040B0021032A08D008E008F11B
:102A8000070020F00702F2E80201904603E080B25E
:102A9000042A00D1C0B24FF0000922072AD53278AB
:102AA000702A07D0DDF800C08CF0100C5CEA0B0C2B
:102AB00005D00EE040228DF80420012208E050EA03
:102AC000010306D030238DF804308DF80520022252
:102AD0009146009B83F0080353EA0B030AD150EAA6
:102AE000010201D1620705D530228DF804204FF094
:102AF00001097F1E3278582A04D039A20C920CAA00
:102B000002920BE03BA2F9E75B46009AFDF793FDCA
:102B10000C9B9B5C029A521E0292137050EA0102B7
:102B2000F2D1029804A9081A00F1200B600702D51F
:102B300024F4803400E001275F4502DDA7EB0B00A1
:102B400000E0002000EB0B01009003984944401A7C
:102B50000390E00306D453462146179A039800F0E9
:102B6000A9F90544002706E001A85246C05D17995F
:102B700090476D1C7F1C4F45F6DBE0030CD5534698
:102B80002146179A039800F095F9054404E0302097
:102B90005246179990476D1C0099481E00900029D5
:102BA000F5DC08E00298029952460078491C02912F
:102BB000179990476D1CBBF10001ABF1010BF1DCE3
:102BC0005BE100F065F90544761C307800287FF45D
:102BD0000DAE19B02846BDE8F08F000009280100AD
:102BE0003031323334353637383961626364656683
:102BF0000000000030313233343536373839414245
:102C00004344454600000000600700D4062708F151
:102C1000070020F00700F0E80223804603F0004C94
:102C20005FEA0C0001D097A009E0200501D596A02D
:102C300005E0E00701D095A001E0AFF24C00139051
:102C4000307823F0004365280CD006DC452809D0F5
:102C500046281DD047287FD13BE0662818D067283A
:102C60007AD136E00021112F01DB112000E0781C21
:102C7000CDE9000104A90CA8FFF7EEFCDDE90D0188
:102C80000C9A4FF0000B07F10109109200914EE0F1
:102C90004FF000400097CDE9011004A90CA8FFF700
:102CA000DBFCDDE90D020C9B0F994FF0000B914608
:102CB0001093009211B9791C00EB0109B7EB0900E0
:102CC00003D4C0F1FF3B07F10109A9EB0700019014
:102CD00042E0012F00DA01270021112F01DD112030
:102CE00000E03846CDE9000104A90CA8FFF7B4FCC8
:102CF000DDE90D010C9A00914FF0000BB9461092DE
:102D000021070FD4009A4A4503DA914601E0A9F160
:102D10000109B9F1010F05DD109AA9F10101515C1A
:102D20003029F4D0B84202DA10F1040F03DA01219D
:102D3000CDE9011010E0002803DC8344A9EB000179
:102D400002E0411C494500DD8946A0EB0B00401C18
:102D500001904FF000400290200705D401984845AB
:102D600002DB4FF0FF30019000208DF84B000298FD
:102D70000DF14B07B0F1004F25D002200C902B2015
:102D80000D90029800280CDA404202902D200D9000
:102D900007E00A210298FDF738FC3031029007F86D
:102DA000011D0C99481E0C900029F2DC02980028A5
:102DB000EFD1791E0D980870307800F0200040F0B7
:102DC000450007F8020D11A8C01BC01D0290139802
:102DD000007800B1012000EB0901019801EBE071DE
:102DE000029801440398401A401E0390E00306D461
:102DF00053462146179A039800F05CF8054413984F
:102E0000007818B15246179990476D1CE00323D5FE
:102E100053462146179A039800F04CF805441BE0EE
:102E2000BBF1000F07DB0098584504DD1098179997
:102E300010F80B0001E01799302052469047019896
:102E40000BF1010B401E05F10105019004D12E206C
:102E50005246179990476D1CB9F10001A9F101097B
:102E6000DEDC05E017F8010B5246179990476D1C00
:102E70000299481E02900029F4DC53462146179A15
:102E800003989EE62D0000002B00000020000000AB
:102E90002DE9F041044600251E461746880404D457
:102EA00005E039462020B0476D1C641EF9D5284640
:102EB000BDE8F0812DE9F041044600251E4690460C
:102EC000C80301D5302700E02027880404D505E099
:102ED00041463846B0476D1C641EF9D52846BDE80A
:102EE000F0814A68002A06D00A68531C0B601070F3
:102EF0004868401E486070470A68531C0B60107099
:102F000070472DE9F84306460F4614464FF0000877
:102F10004FF00409FF2249466846FDF763F924F0A3
:102F200003052DB12A463946304601F06BF980463B
:102F3000651BB8F1000F0FD175B124F00300C11962
:102F40002A466846FDF73CF924F0030188194A46F1
:102F5000694601F057F980464046BDE8F883000015
:102F600013B586B004464FF0FF3005900020049062
:102F700003901C4903AB04AACDE90010014620468A
:102F800003F0C6FA039848B10120174905AB07AA18
:102F9000CDE900100221204603F0BAFA0498002877
:102FA0001DD00598401C002819D10498012802D88A
:102FB0000E48007850B101200B4905AB07AACDE9B6
:102FC00000100146204603F0A3FA08E008A240F2F0
:102FD000254112A001F042F801200449087005982B
:102FE00008B010BD716500083D300008E9010020FF
:102FF0005472696767657220612047432063686582
:10300000636B20616674657220616C6C6F63204530
:103010004E56206661696C65642E0A002E2E5C2E69
:103020002E5C557365725C6561737964625C737262
:10303000635C65665F656E762E63000070B503465F
:103040000C461546187880B118692668B0420CD92C
:103050009878012805D09878022806D1044800788D
:1030600018B958692860012070BD0020FCE70000F5
:10307000E901002010B504462078C0F3430020B1D8
:10308000012803D0052819D117E017E002F0F8FF56
:10309000808A00F4007078B102F0F2FF00218171A3
:1030A00002F0EEFF0121C17102F0EAFF002101717F
:1030B00002F0E6FF0121417100E000BF00BF10BD3A
:1030C00010B504462078C0F3430020B1012803D096
:1030D000052839D137E037E002F0D2FF808A00F4CA
:1030E000806078B302F0CCFF0021817102F0C8FF4C
:1030F0004078012811D102F0C3FF007801280CD1DB
:1031000001021248FEF735FB11484168002088474C
:1031100002F0B6FF0021417014E002F0B1FF4078E8
:1031200080B902F0ADFF007801280BD101020748F9
:10313000FEF721FB064841680020884702F0A0FF07
:103140000121417000E000BF00BF10BD000C014034
:103150002C00002010B504462078C0F3430020B1B5
:10316000012803D005280BD109E009E002F088FF0F
:103170000021817102F084FF0121017200E000BF93
:1031800000BF10BD70B504462078C0F3430020B1E5
:10319000012803D005282AD124E028E002F070FF9E
:1031A000007808B9012500E0002502F069FF0570EC
:1031B00002F066FF002181710E48416800208847B7
:1031C00002F05EFF0021C17102F05AFF002101727E
:1031D0004FF480710848FEF7CCFA02F051FF00214D
:1031E000417004E002210548FEF7C3FA00BF00BFAA
:1031F00070BD00002C000020000C014000080140C0
:1032000010B504462078C0F3430020B1012803D054
:10321000052815D113E013E002F032FF007D00F025
:10322000020058B102F02CFF0021817102F028FF4A
:103230000121C17002F024FF0121C17100E000BF33
:1032400000BF10BD10B504462078C0F3430020B184
:10325000012803D0052815D113E013E002F010FF78
:10326000007D00F0040058B102F00AFF00218171D6
:1032700002F006FF0121C17102F002FF03218170FB
:1032800000E000BF00BF10BD10B504462078C0F3B9
:10329000430020B1012803D0052815D113E013E025
:1032A00002F0EEFE007D00F0080058B102F0E8FEEA
:1032B0000021817102F0E4FE0121C17102F0E0FE03
:1032C0000421817000E000BF00BF10BD10B50446AE
:1032D0002078C0F3430020B1012803D0052815D180
:1032E00013E013E002F0CCFE007D00F0100058B1B6
:1032F00002F0C6FE0021817102F0C2FE0121C171FF
:1033000002F0BEFE0521817000E000BF00BF10BDCD
:1033100010B504462078C0F3430020B1012803D043
:10332000052815D113E013E002F0AAFE007D00F09D
:10333000200058B102F0A4FE0021817102F0A0FE2D
:103340000121C17102F09CFE0621817000E000BFE6
:1033500000BF10BD10B504462078C0F3430020B173
:10336000012803D0052815D113E013E002F088FEF0
:10337000007D00F0400058B102F082FE0021817112
:1033800002F07EFE0121C17102F07AFE07218170F8
:1033900000E000BF00BF10BD10B504462078C0F3A8
:1033A000430020B1012803D0052815D113E013E014
:1033B00002F066FE007D00F0800058B102F060FE71
:1033C0000021817102F05CFE0121C17102F058FE02
:1033D0000821817000E000BF00BF10BD10B5044699
:1033E0002078C0F3430020B1012803D0052819D16B
:1033F00017E017E002F044FE808A00F4807078B194
:1034000002F03EFE0021817102F03AFE0121C171FD
:1034100002F036FE0121017102F032FE00214171FD
:1034200000E000BF00BF10BD10B508210148FEF745
:1034300097F910BD000C014010B502210148FEF7BC
:103440008FF910BD000C014010B54FF480510248B7
:10345000FEF786F910BD0000000C014010B50121F7
:103460000148FEF77DF910BD0008014010B54FF48A
:1034700000610248FEF774F910BD00000008014029
:1034800010B54FF480510248FEF76AF910BD0000F4
:103490000008014010B580210148FEF761F910BD18
:1034A000000C014010B54FF480410248FEF758F976
:1034B00010BD0000000C014010B540210148FEF78E
:1034C0004FF910BD000C014010B54FF400510248F7
:1034D000FEF746F910BD0000000C014010B5202198
:1034E0000148FEF73DF910BD000C014010B54FF446
:1034F00000410248FEF734F910BD0000000C014005
:1035000070B586B004460D461646607800281DD07A
:10351000207803281AD1A17804F11002124800F093
:10352000C9FD204601F08EFE30B910A240F2BD6107
:1035300016A000F093FD15E01C4A40F2BF6113A0F5
:10354000A36800F08BFD012006B070BD2078012833
:1035500007D10523062201A9206B05F0DBFB012022
:10356000F2E700BF0020EFE754A200085265636F46
:10357000766572792074686520454E5620737563B0
:103580006365737366756C2E0A0000002E2E5C2E28
:103590002E5C557365725C6561737964625C7372ED
:1035A000635C65665F656E762E630000F0A20008BE
:1035B00070B504460D461646207838B1A078032829
:1035C00004D101200249087001F0D2F9002070BD39
:1035D000E90100202DE9F04104460D461746207808
:1035E00068B92E460748616800F064FD3068401CE9
:1035F00030604FF0FF31606801F02EF900BF00200D
:10360000BDE8F08110A200082DE9F04389B004461E
:103610000D460027A1461DE004F12000A84202D279
:103620004FF0200801E0A5EB0408424601A920461E
:1036300000F0DAFD00260AE0FF2F05D001A8805D2A
:10364000FF2801D104EB060901A8875D761C4645D9
:10365000F2D32034AC42DFD3FF2F06D109F10300AF
:1036600020F0030009B0BDE8F0832846FAE7000027
:103670002DE9F0478CB00646884691469A460024CC
:103680000020019075694046FCF7CAFD202807D943
:10369000202164A000F00EFD04200CB0BDE8F087EE
:1036A000FF22282102A8FCF79DFD694807904046AB
:1036B000FCF7B6FDC0B28DF82800CDF82CA09DF81F
:1036C0002800C01C20F0030128310B98C01C20F0FA
:1036D0000300084408900898B0F5777F04D95DA0EE
:1036E00000F0E8FC0620D8E7681C38B93046089995
:1036F00001F060FE0546401C00287DD02CB901AACF
:103700003046089904F080FC0446002C3ED1FF208E
:10371000009008220AA9002000F06AFA09909DF89A
:1037200028204146099800F063FA09909DF8280086
:10373000C01C20F003009DF82810471A05E0012264
:103740006946099800F054FA0990381EA7F101075C
:10375000F5D149460B9A099800F04AFA09900B985E
:10376000C01C20F003000B99471A05E001226946AE
:10377000099800F03DFA0990381EA7F10107F5D12C
:1037800002A9284605F0AEFA044600BF04BB9DF826
:103790002820414605F12800FFF7B3FB04469DF8B9
:1037A000040078B99DF82820D21C22F0030305F10B
:1037B000280213440B9AD21C22F003029918706855
:1037C00004F052FC9DF828102A46404604F09AFB6B
:1037D00064B99DF82810C91C21F0030305F12801E4
:1037E000581849460B9AFFF78CFB044644B902234C
:1037F000062202A9284600E010E005F08BFA0446F4
:103800005CB99DF8040040B11AA240F25E5123A0B9
:1038100000F024FC01202949087000E0062420461D
:103820003BE700004572726F723A2054686520458C
:103830004E56206E616D65206C656E6774682069F8
:1038400073206D6F7265207468616E2025640A00B4
:103850004B5634304572726F723A20546865204579
:103860004E562073697A6520697320746F6F2062E9
:1038700069670A005472696767657220612047436F
:1038800020636865636B206166746572206372658E
:103890006174656420454E562E0A00002E2E5C2E63
:1038A0002E5C557365725C6561737964625C7372DA
:1038B000635C65665F656E762E630000E90100203B
:1038C0002DE9F04393B005460C461746002694B9FF
:1038D0006946284600F04BFD08B16C460AE02B46CD
:1038E00027A240F23F412CA000F0B8FB042013B007
:1038F000BDE8F08300BF57B9032306220EA9206B51
:1039000005F008FA064601202B49087021E004233F
:1039100006220EA9206B05F0FDF906462648007820
:10392000A0B99EB955B12846FCF77AFC81464FF004
:10393000FF324946284604F0E5FA07E034B1A178A1
:103940004FF0FF3204F1100004F0DCFA00201A49B5
:103950000870206B6FF3090000F10C086EB90422A7
:103960000EA9404602F08CFD012806D10223042254
:103970000EA9404605F0CEF906463046B7E70000EE
:103980004E6F7420666F756E64202725732720693B
:103990006E20454E562E0A002E2E5C2E2E5C557340
:1039A00065725C6561737964625C7372635C6566A1
:1039B0005F656E762E630000EB01002010B56FF09E
:1039C0000400FEF763FA0A4800680A49B0FBF1F008
:1039D000094908700846007800EB4001C1EBC010AF
:1039E0004FF6FF7101EAC0000449088010BD0000D5
:1039F000C401002000127A0064000020660000204C
:103A00000146114A12884A434FF0E0235A610022CE
:103A10009A611A46126942F001021A6100BF4FF022
:103A2000E022106900F001021AB100F48032002A8D
:103A3000F5D04FF0E022126922F001024FF0E023AE
:103A40001A6100229A6170476600002070B592B03A
:103A500004460D4616462078002842D0A078022859
:103A600002D0A07803283CD1616801F10C00032347
:103A7000042201A905F04EF94FF0FF3010901BE031
:103A800004A802F001FB9DF81100A8B19DF81000F8
:103A9000022803D09DF8100003280DD104A801F0DE
:103AA000D1FB48B108A800909DF812300EA240F258
:103AB000D94118A000F0D2FA04A9204601F068F913
:103AC0001090401C0028DBD14FF0FF31606800F0FF
:103AD000C3FE18A240F2DE410EA0636800F0BEFAF9
:103AE00000BF002012B070BD4572726F723A204D57
:103AF0006F7665642074686520454E562028252E13
:103B00002A732920666F72204743206661696C65BD
:103B1000642E0A002E2E5C2E2E5C557365725C6539
:103B200061737964625C7372635C65665F656E760F
:103B30002E630000436F6C6C6563742061207365B5
:103B400063746F7220403078253038580A000000C6
:103B50001CB50020019000240F48007808B1002017
:103B60001CBD01A9684600F035FB044624B9DDE917
:103B7000000100F053F804463CB9012006490870E2
:103B800006A108A000F096FA03E004A10FA000F03F
:103B900091FA2046E4E70000D8010020342E312EAF
:103BA0003939000045617379466C61736820562588
:103BB0007320697320696E697469616C697A652024
:103BC000737563636573732E0A0000004561737932
:103BD000466C6173682056257320697320696E698D
:103BE0007469616C697A65206661696C2E0A0000EF
:103BF00030B503460C46DB4308E014F8010B58408F
:103C0000C0B2054D55F8200080EA1323101EA2F122
:103C10000102F2D1D84330BDC49B0008F8B5054677
:103C20000E46002755B91F481FA322A240F2067175
:103C3000009028A000F012FA00BFFEE72D4800789F
:103C400008B10020F8BD002405E04FF0FF302A49FC
:103C500041F83400641C042CF7D3002406E04FF034
:103C6000FF30264901EBC4014860641C102CF6D3D8
:103C700023482449086024480560244806604FF41E
:103C800000601F4B22A24FF4E461009011A000F0ED
:103C9000E5F900F07DF9074617B9012015490870CC
:103CA0003846CFE7B79B000864656661756C745F42
:103CB000656E76002825732920686173206173730F
:103CC000657274206661696C656420617420257377
:103CD0002E0A00002E2E5C2E2E5C557365725C65DC
:103CE00061737964625C7372635C65665F656E764E
:103CF0002E630000E801002034360020B435002097
:103D000000DC0008DC010020E0010020E4010020CC
:103D1000454E5620737461727420616464726573D9
:103D200073206973203078253038582C2073697AD5
:103D3000652069732025642062797465732E0A00FA
:103D4000F0B587B000263748006850B9364837A329
:103D50003AA240F20961009040A000F07FF900BF54
:103D6000FEE74648006850B92F4845A333A240F209
:103D70000A61009039A000F071F900BFFEE700F081
:103D8000BBF94548056809E04FF0FF31284600F0CF
:103D900063FD064606B13FE005F580653E480068D4
:103DA00000F500608542EFD3002430E004EB4400CE
:103DB0001C49096801EB8000806850B904EB44019C
:103DC000184A126802EB81014868FCF729FA074695
:103DD00006E004EB44001349096801EB80008768A2
:103DE0004FF0FF30069004EB44000E4B1B6803EBD2
:103DF0008000426804EB44000A4B1B6853F8201013
:103E00003B4601A8FFF734FC06B105E0641C1B48E3
:103E100000688442CAD300BF00F070F9304607B092
:103E2000F0BD0000E0010020A49B0008646566610D
:103E3000756C745F656E765F7365740028257329F1
:103E40002068617320617373657274206661696CA8
:103E500065642061742025732E0A00002E2E5C2ECE
:103E60002E5C557365725C6561737964625C737214
:103E7000635C65665F656E762E630000E40100207A
:103E800064656661756C745F656E765F7365745F9B
:103E900073697A6500000000DC01002070B50546FA
:103EA000002380220B49284600F034F8041E0ED06F
:103EB0002146084800F05CF820B10020054908556B
:103EC000084670BD04A000F0F5F80020F9E70020D6
:103ED000F7E70000543600205761726E696E673A4A
:103EE0002054686520454E562076616C75652069C2
:103EF000736E277420737472696E672E20436F751A
:103F00006C64206E6F742062652072657475726EC9
:103F100065640A002DE9F04104460D4616461F4629
:103F20004FF000080A48007828B90AA000F0C2F84B
:103F30000020BDE8F08100F0DFF83B46324629461C
:103F4000204600F0ADFE804600F0D8F84046F0E78D
:103F5000E8010020454E562069736E277420696E73
:103F6000697469616C697A65204F4B2E0A00000004
:103F700002460B46002106E0505C20385F2801D342
:103F800000207047491C9942F6D30120F9E7000050
:103F900010B598B000240020039001201A49087041
:103FA00000201A49034603AACDE90010014604A8DF
:103FB00002F0AEFA0398022804D115A000F07AF8B6
:103FC000FFF7BEFE00F098F80020214903460246A4
:103FD000CDE90010014604A802F09AFA00BF1D4B7B
:103FE000002211460AA800F085F91B48007810B19C
:103FF00000F0BEFCF3E700200349087000F07EF8F3
:10400000204618B010BD0000EA010020D535000898
:104010005761726E696E673A20416C6C20736563FC
:10402000746F722068656164657220636865636B94
:10403000206661696C65642E205365742069742064
:10404000746F2064656661756C742E0A0000000050
:10405000B135000801350008E90100200FB438B57A
:1040600004460D4607A800902A46214609A000F004
:10407000EFF80D48009A0699FEF7C8FA0A490BA016
:1040800000F0E6F80AA0FEF783FA0020009038BCA2
:104090005DF814FB5B466C6173685D2825733A25F7
:1040A0006C642920000000002837002025730000E0
:1040B0000D0000000FB408B503A8009009A000F09F
:1040C000C7F80A48009A0299FEF7A0FA074908A023
:1040D00000F0BEF807A0FEF75BFA0020009001B0E8
:1040E0005DF814FB5B466C6173685D002837002047
:1040F000257300000D00000072B6704762B670476D
:104100002DE9F84305460E464FF00009C5F30900B6
:1041100048B1164816A31EA26121009024A0FFF703
:104120009DFF00BFFEE74FEA9628C6F3090008B1DD
:1041300008F10108FDF722FA3520FDF799F900246E
:104140000CE04FF4806101FB0450FDF797F907463E
:10415000042F02D04FF0010902E0641C4445F0D363
:1041600000BFFDF7CBF94846BDE8F883D09F0008B3
:104170006164647220252045465F45524153455F86
:104180004D494E5F53495A45203D3D2030000000C7
:104190002825732920686173206173736572742008
:1041A0006661696C65642061742025732E0A0000C5
:1041B0002E2E5C2E2E5C557365725C65617379647E
:1041C000625C706F72745C65665F706F72742E6390
:1041D0000000000002460020024B136001230B6028
:1041E00070470000C49F000870B5034600200C46CD
:1041F000002504E01E7826706D1C5B1C641C954233
:10420000F8D370BD2DE9F04705460C4616464FF031
:104210000009FDF7B3F93520FDF72AF900270EE074
:1042200028462168FDF774F9D5F8008020684045DC
:1042300002D04FF0030904E03F1D241D2D1DB7429D
:10424000EED300BFFDF75AF94846BDE8F0870000FD
:104250000FB408B503A800900648009A0299FEF72B
:10426000D5F9044904A0FEF793F90020009001B0AD
:104270005DF814FB283700202573000000207047EC
:1042800070B505460C462046FBF7CAFF0646324687
:104290002146284600F002F870BD00002DE9F041EB
:1042A00004460D46164600270A48007828B90AA099
:1042B000FFF700FF0720BDE8F081FFF71DFF324642
:1042C0002946204602F06CF90746FFF717FF3846EB
:1042D000F1E70000E8010020454E562069736E2783
:1042E0007420696E697469616C697A65204F4B2E20
:1042F0000A0000002DE9F04186B004460E4617463C
:104300001D464FF0FF30019028E0002269464046EC
:1043100001F0C0FF00B121E005B91FE09DF80100E8
:10432000022803D09DF80100032816D14FF0FF307A
:1043300020630AE0204601F0A7FE3A4631462046B7
:10434000A84710B106B0BDE8F0812146684600F0EC
:104350001FFD2063401C0028ECD100BF684600F020
:104360004DFD8046401C0028CFD100BFEAE72DE973
:10437000F04106460C4600253046FBF751FF074644
:1043800004F130023946304600F0AEFC28B1204638
:1043900001F07AFE0120BDE8F0812146304600F0B0
:1043A0002DF8054625B139463046226B03F0AAFDAB
:1043B0002846F0E72DE9F04704460D4616462F46FD
:1043C000B1463846FBF72CFF8046A078404502D026
:1043D0000020BDE8F087607868B1207802280AD113
:1043E0004246394604F11000FBF72FFF18B90120AF
:1043F00089F80000EDE70020EBE7000038B504463F
:104400000D4600200090044B6A4621462846FFF7DF
:1044100071FF9DF8000038BDB54300082DE9F0415B
:104420008AB004460E462746A00A800201A900F081
:1044300005FD38B10198844204D14FF0FF300AB035
:10444000BDE8F08126E0202202A92046FFF7CCFE3D
:10445000002519E002A8415D02AA681C105C01EB6E
:104460000021A81C105C01EB0041E81C105C01EB72
:1044700000680B48804506D160191438B84202D351
:1044800060191438DBE76D1C1C2D02D26019B04294
:10449000E0D31C34B442D6D34FF0FF30CFE7000056
:1044A0004B56343070B50025A748046800BF47E17B
:1044B00020784009002802DD6088401C6080207858
:1044C0004009072822D2DFE800F0042246C9E5F2BD
:1044D000F1000120A8409D490988084088B10020CA
:1044E0006080A080207820F0E000203020702078CC
:1044F00020F01E002070606940B120466169884745
:1045000004E0207820F01E001430207014E1012017
:10451000A8408F490988084028B9207820F0E00099
:104520004030207016E060886189884212DB608824
:10453000A18988420EDA207820F0E00080302070D7
:10454000207820F01E00801D2070606910B1204688
:1045500061698847F0E06088218988421DDAA08877
:10456000401CA080A088012805D1207820F0E00020
:104570006030207071E00020A080207820F0E00002
:104580002070207820F01E00001D20706069002837
:1045900063D02046616988475FE06088218988424E
:1045A00015DB60886189884211DA0020A0802078BC
:1045B00020F0E0002070207820F01E00801C207089
:1045C0006069002849D020466169884745E06088D5
:1045D0006189884214DB6088A189884210DA002052
:1045E000A080207820F0E0002070207820F01E00CD
:1045F00008302070606980B32046616988472CE0EC
:104600006088A189884214DB6088E189884210DAD9
:104610000020A080207820F0E0002070207820F09A
:104620001E000C3020706069B8B12046616988476F
:1046300013E06088E18988420FDB0020A0802078A9
:1046400020F0E0002070207820F01E001030207054
:10465000606910B12046616988476DE00120A8407B
:104660003A490988084058B1A088401CA0802078A9
:1046700020F0E000403020706088401E608008E03C
:1046800060882189884204DB207820F0E0004030F7
:10469000207051E00120A8402D490988084038B910
:1046A000207820F0E0004030207018E038E017E07B
:1046B0006088A189884212DB6088E18988420EDA2D
:1046C000207820F0E000A0302070207820F01E003C
:1046D0000A302070606910B12046616988472BE07C
:1046E0000120A8401A490988084028B9207820F0FC
:1046F000E0004030207012E06088E18988420EDBE3
:10470000207820F0E000C0302070207820F01E00DB
:104710000E302070606910B12046616988470BE057
:104720000120A8400A490988084020B9207820F0D3
:10473000E0004030207000BF00BFA469681C45B293
:10474000002C7FF4B5AE70BD680000206C00002026
:104750006E00002070B500251948008819490880AE
:1047600000261948046800BF16E0207800F0010018
:1047700038B12069804708B9012000E00020B0402E
:1047800002E020698047B0400E49098808430D497E
:104790000880A469701C46B214B120690028E4D1D5
:1047A000084800884FF6FF7180EA0105074909882B
:1047B00085EA01002840064908800448058070BD4C
:1047C0007200002070000020680000206E000020B1
:1047D0006C00002001461A48026819B11948007897
:1047E000102802DD4FF0FF30704705E08A4202D109
:1047F0004FF0FF30F8E79269002AF7D110480068BF
:104800008861087820F0E0000870087820F01E0029
:1048100014300870002048808880094801600A48E8
:1048200000884FF6FF7303EA4000074B18800548E5
:104830000078401C034B18701846007840B2D3E74C
:1048400068000020740000207200002010B5FFF7FF
:1048500081FFFFF727FE10BD70B58AB004460D46F4
:104860000026C4F3090050B11A481BA320A240F24D
:10487000AD31009026A0FFF7F1FB00BFFEE74FF43B
:1048800080612046FFF73CFC0646FEB9FF2224214A
:1048900001A8FBF7A7FC0122042101A801F0CAFE30
:1048A0000122042104A801F0C5FE214807900895C3
:1048B0004FF0FF300990242201A92046FFF7A2FC07
:1048C000064604F58061204603F0CEFB30460AB070
:1048D00070BD0000969B000861646472202520531F
:1048E0004543544F525F53495A45203D3D203000C7
:1048F00028257329206861732061737365727420A1
:104900006661696C65642061742025732E0A00005D
:104910002E2E5C2E2E5C557365725C656173796416
:10492000625C7372635C65665F656E762E63000021
:104930004546343070B504460D46E1B20548FDF7F2
:1049400092FD00BF80210348FDF7BFFC0028F9D08D
:10495000204670BD0038014010B5034614460A4693
:10496000187810B11068401C1060002010BD0000C5
:1049700000B589B0002002901149034602AACDE992
:104980000010012103A801F0C3FD012000900DA239
:1049900040F2F24118A0029BFFF760FB0298012849
:1049A00009D800201C4903460246CDE90010014603
:1049B00003A801F0ADFD00201849087009B000BD42
:1049C000594900085468652072656D61696E2065FB
:1049D0006D70747920736563746F7220697320251C
:1049E000642C204743207468726573686F6C642080
:1049F00069732025642E0A002E2E5C2E2E5C5573C2
:104A000065725C6561737964625C7372635C656630
:104A10005F656E762E6300004D3A0008E9010020C4
:104A20002DE9FE4F824600200290BAF10A0F23D2F0
:104A3000DFE80AF00523405D7A97B4D1F0EE94499F
:104A40000888FBF7B1FD8346FBF7CCFD4FF06632DB
:104A5000904BCDE90001FBF7BDFC804600228E4B58
:104A6000FBF7B8FC064600228C4BFBF725FD0446FD
:104A7000FBF79FFD80B2029006E185494888FBF76D
:104A800093FD4FF08B410190FBF766FC8346FBF7EB
:104A9000A9FD80464FF066327E4BFBF79BFC064635
:104AA00000227D4BFBF796FC0446FBF782FD80B2AB
:104AB0000290E9E076498888FBF776FD4FF08B415C
:104AC0000190FBF749FC8346FBF78CFD80464FF0D5
:104AD0006632704BFBF77EFC064600226E4BFBF7FE
:104AE00079FC0446FBF765FD80B20290CCE0684992
:104AF000C888FBF759FD4FF08B410190FBF72CFC68
:104B00008346FBF76FFD06464FF06632614BFBF7BD
:104B100061FC80460022604BFBF75CFC0446FBF71F
:104B200048FD80B20290AFE059490889FBF73CFD8F
:104B30004FF08B410190FBF70FFC8346FBF752FDD2
:104B400080464FF06632534BFBF744FC064600228A
:104B5000514BFBF73FFC0446FBF72BFD80B2029064
:104B600092E04B494889FBF71FFD4FF08B410190C4
:104B7000FBF7F2FB8346FBF735FD80464FF06632CC
:104B8000444BFBF727FC06460022434BFBF722FC75
:104B90000446FBF70EFD80B2029075E03C4988891F
:104BA000FBF702FD4FF08B410190FBF7D5FB8346ED
:104BB000FBF718FD80464FF06632364BFBF70AFCD8
:104BC00006460022344BFBF705FC0446FBF7F1FCDC
:104BD00080B2029058E02E49C889FBF7E5FC4FF0FF
:104BE0008B410190FBF7B8FB8346FBF7FBFC0646C5
:104BF0004FF06632274BFBF7EDFB80460022264B39
:104C0000FBF7E8FB0446FBF7D4FC80B202903BE0E4
:104C10001DE0FFE71E49088AFBF7C6FC4FF08B41F9
:104C20000190FBF799FB8346FBF7DCFC06464FF04F
:104C30006632184BFBF7CEFB80460022164BFBF783
:104C4000C9FB0446FBF7B5FC80B202901CE010499A
:104C5000488AFBF7A9FC4FF08B410190FBF77CFBE6
:104C60008346FBF7BFFC06464FF06632094BFBF765
:104C7000B1FB04460022084BFBF7ACFB8046FBF778
:104C800098FC80B2029000BF00BF0298BDE8FE8F82
:104C90005003002066660A40000059400000B04002
:104CA0002DE9F0418EB080460E4615461C46002781
:104CB00069464046FFF75BFB78B10CB10398206072
:104CC0000398A84201D2039F00E02F4646B13A461E
:104CD00031460D98FFF788FA02E00CB10020206001
:104CE00038460EB0BDE8F0812DE9F04188B00546A8
:104CF0000E461746324629460020FEF779FF4FEA56
:104D0000104800243EE0214800EBC4004068401CED
:104D1000A8B31E4830F83400404532D11B4901EB9E
:104D2000C401496801F1280020226946FFF75CFAB6
:104D3000324669462846FBF788FA08BB134800EB61
:104D4000C40040683860114800EBC40040884FF64A
:104D5000EF71884206DB4FF6FF700C4901EBC4018E
:104D6000488008E0094800EBC4004088103007493B
:104D700001EBC4014880012008B0BDE8F08100E0EB
:104D800000BF641C102CBED30020F5E7B435002012
:104D900070B505460C464FF0FF366878012801D102
:104DA000801E70BD206B401C18B9686800F1240695
:104DB00021E0216B686800F58060814218D8607836
:104DC00018B1A168206B461801E0206B061D6868C9
:104DD00000F577713046FFF721FB0646686800F55D
:104DE0008060B04201D3A06828B94FF0FF30D8E707
:104DF0004FF0FF30D5E73046D3E700000146486862
:104E0000401C10B90C4800687047C868401C18B9AD
:104E1000486800F5806203E04B68C86803EB8022B5
:104E20000548006800F50060824201D21046EBE7B9
:104E30004FF0FF30E8E70000DC01002003460A469F
:104E400000210DE0084850F83100984207D122B106
:104E5000054800EBC1004068106001207047491C04
:104E60000429EFD30020F9E73436002030B502469C
:104E70000023481E0146044606E0480102EBD0002C
:104E8000007800B904E05B1C081EA1F10101F4D117
:104E900000BFE01A30BD000070B501F059FF0646B2
:104EA00001F0EEF8848A214641A0FDF771FB01F084
:104EB000E7F8007D00F0020008B146A000E047A03E
:104EC0000446214647A0FDF763FB01F0D9F8007DB9
:104ED00000F0080008B13FA000E040A0044601F047
:104EE000CFF8007D00F0040008B13AA000E03BA03C
:104EF00005462246294640A0FDF74AFB01F0C0F8CE
:104F0000007D00F0200008B132A000E033A004468C
:104F100001F0B6F8007D00F0100008B12DA000E00F
:104F20002EA005462246294637A0FDF731FB01F0A9
:104F3000A7F8007D00F0800008B126A000E027A0BF
:104F4000044601F09DF8007D00F0400008B121A06A
:104F500000E022A00546224629462FA0FDF718FBB7
:104F600001F08EF8808A00F4007008B119A000E00A
:104F70001AA0044601F084F8808A00F4807008B119
:104F800014A000E015A005462246294626A0FDF7FC
:104F9000FFFA01F075F8808A00F4806008B10DA076
:104FA00000E00EA00446214623A0FDF7F1FA70BDF3
:104FB000E5BD93E5898DE68C89E994AEE4BDBFE853
:104FC00083BDE78AB6E680813A20307825303458B0
:104FD0000D0A0000E4BDBFE883BD0000E5A4B1E810
:104FE00083BD000030312E4E554C4C202030322EE7
:104FF00025730D0A0000000030332E257320203069
:10500000342E25730D0A000030352E2573202030F4
:10501000362E25730D0A000030372E2573202030E0
:10502000382E25730D0A000030392E2573202031CB
:10503000302E25730D0A000031312E2573202031CA
:10504000322E4E554C4C0D0A000000002DE9FC415B
:1050500005460C4601F07CFE0746022D32DB0B2D87
:1050600030DC012C01D0002C2CD154B101F008F817
:1050700000F11406808A691E01228A4010433080A4
:1050800009E000F0FDFF00F11406808A691E01228C
:105090008A409043308000F0F3FF868A33461FA297
:1050A00006216846FDF784FA69461EA0FFF7E8F876
:1050B0000CB120A000E021A00246294621A0FDF766
:1050C00067FA29E0002D24D1012C01D0002C20D139
:1050D0002CB100F0D5FF4FF6FF71818203E000F0A4
:1050E000CFFF0021818200F0CBFF868A33460BA2DE
:1050F00006216846FDF75CFA69460AA0FFF7C0F88A
:105100000CB10CA000E00DA0014615A0FDF740FA7F
:1051100002E01AA0FDF73CFABDE8FC813078255882
:10512000000000006B65795F656E5F7461626C659D
:1051300000000000E4BDBFE883BD0000E5A4B1E8C5
:1051400083BD0000E68C89E994AE2564E68890E58D
:105150008A9FE8AEBEE7BDAE2573200A00000000BE
:10516000E68980E69C89E68C89E994AEE68890E53C
:105170008A9FE8AEBEE7BDAE25730A0020E8AEBE4A
:10518000E7BDAEE5A4B1E8B4A5EFBC8CE8AFB7E6E7
:10519000A380E69FA5E58F82E695B0200A00000077
:1051A00070B594B0044601F0D3FD06465021684620
:1051B000FBF71FF820783F2801D114B070BD2246BC
:1051C00009A16846FDF70EFA6846FBF729F885B293
:1051D00007482A466946C368064898474FF49670C0
:1051E00003F0B4FA00BFE8E741542B25730D0A0021
:1051F00044000020004800401CB50124FBF772FF6A
:105200000A48012100234A02CDE9001008A10C48F8
:1052100004F09AF90446012C02D103F047FC02E0A5
:105220004FF0FF301CBD00BFFEE700000000002073
:105230004170705461736B43726561746500000066
:10524000410E00082DE9F043A3B004464FF00009D9
:105250002078022804D1002221461046FEF730FBB8
:1052600018A8A168FDF77CFE0546401CA8B13C4883
:105270000078B0B1242101A8FAF7BBFFA27804F1AD
:10528000100101A8FAF7C0FF0AA901A8FFF7B6F8B4
:1052900010B14FF000095CE003E0062023B0BDE848
:1052A000F083A768002218A8A16802F0ADFE0123D0
:1052B00006221EA9284603F02DFD143F0026B04605
:1052C0001BE006F12000B84202D24FF0200801E0B6
:1052D000A7EB060808F1030121F00302216B14314A
:1052E000881910A9FEF780FF05F1140188194246BC
:1052F00010A9FEF787FF81464644BE42E1D3022350
:1053000006221EA9284603F005FDA278D21C22F031
:10531000030305F128021344E268D21C22F00302C1
:105320009918A80A800202F09FFEA1782A4604F18B
:10533000100002F0E7FD04F11001206BCDE901053A
:105340000091A37807A240F29E4112A0FEF786FECC
:1053500000BF012221460020FEF7B2FA48469DE731
:10536000EA0100204D6F7665642074686520454E23
:10537000562028252E2A73292066726F6D203078DA
:105380002530385820746F203078253038582E0A50
:10539000000000002E2E5C2E2E5C557365725C653D
:1053A00061737964625C7372635C65665F656E7677
:1053B0002E6300002DE9F04105460C460026771EBD
:1053C00000BF21462846FDF7CBFD0746401C70B9BB
:1053D0000848007858B156B92346074A40F2AE4112
:1053E00006A0FEF73BFEFFF7C3FA0126E9E73846C1
:1053F000BDE8F081E9010020A0A200082E2E5C2E5D
:105400002E5C557365725C6561737964625C73725E
:10541000635C65665F656E762E6300002DE9F04182
:1054200006460C461546E01C20F003012831E81C16
:1054300020F003000F1839463046FFF7BBFFBDE8E8
:10544000F08100002DE9F04105460E461C48076832
:105450001C480068001D02F0C1FF50B919480068DF
:1054600090F82C100120884017490968814316489C
:105470000160681C38B936B112480168091D13482B
:1054800002F0EAFF1AE07C190E4800684460BC4252
:1054900007D20C480168091D0D48006802F0C2FFE0
:1054A0000CE008480168091D0A48006802F0BAFFCC
:1054B00009480068844201D207480460BDE8F081D1
:1054C000500100203C01002054010020780D0020F4
:1054D00044010020400100206C01002010B504466A
:1054E00002F0C6FF23480068401C22490860224899
:1054F000006840B9204804600846006801280DD1C2
:1055000000F02CFA0AE01D48006838B91A48006813
:10551000C06AE16A884201D81748046018480068E8
:10552000401C1749086094F82C1001208840154948
:105530000968084313490860E16A01EB8101124AD6
:1055400002EB8100211D02F087FF02F0D3FF0B4820
:10555000006868B108480068C06AE16A884207D2FA
:105560004FF0805009490860BFF34F8FBFF36F8F32
:1055700010BD00004C0100203C010020580100201B
:105580006801002054010020A80A002004ED00E07A
:1055900010B502F06DFF10480068D0B90F4802F056
:1055A00031FF0F4802F02EFF0C480E4908600C48EE
:1055B0000D49086000220C210A2003F095FC0649E1
:1055C00008600846006820B108A10348006803F09D
:1055D00081F802F08FFF10BD800100208C0D0020AB
:1055E000A00D0020780100207C010020546D725134
:1055F0000000000070B523E003F0B2FA1348006821
:1056000008B9012000E00020054604F065F9BDB9A5
:1056100002F02EFF0D48C068C468201D02F0DEFEB7
:105620000B480068401E0A4908600A480068401E8E
:105630000849086002F05EFF204600F060F800BFF5
:10564000044800680028D7D170BD0000640D002018
:105650004C0100204801002070B504460D46206C26
:1056600070B1216CE0680844E0606168E0688842DD
:1056700001D32068E0602846226CE168FAF7A0FDBB
:1056800070BD2DE9F04104460F4615464FF0000865
:10569000A66B206C40B9206860BB606804F04EF8CF
:1056A00080460020606025E07DB93946226CA06804
:1056B000FAF786FD216CA0680844A060D4E90110C7
:1056C000884217D32068A06014E03946226CE06855
:1056D000FAF776FD216CE068401AE0602168E06826
:1056E000884203D2216C6068401AE060022D01D12B
:1056F00006B1761E701CA0634046BDE8F08110B56F
:105700000446206B02F02CFF204602F029FF10BD5A
:105710000146084A126812680AB9012200E0002214
:105720000A600A6822B9034A1268D268106800E069
:10573000002070477801002030B54FF420531748FF
:1057400000F007042CB1C01D20F00700134C041B0F
:105750001B1B0246124C22600024114D6C60D018B5
:10576000083820F007000F4C206000240D4D2D68F4
:105770006C600C4D2D682C601146441A4C60094C2D
:1057800024680C60084D4C682C60084D4C682C60F7
:105790004FF00044064D2C6030BD0000B40D0020D9
:1057A0008C010020940100209C0100209801002021
:1057B000A001002000BFFFF71DFF06480068012878
:1057C000F9D94FF0805004490860BFF34F8FBFF301
:1057D0006F8FF0E7A80A002004ED00E010B5044642
:1057E0004CB1002060602060E06000231A4619463A
:1057F000204603F0FBFC10BD2DE9F04106460D46A6
:1058000017469846069C0DB9246000E02760E663C1
:1058100025640121204603F08DFCBDE8F0810000E5
:105820002DE9FF5F81460F469246DDE90E6B109C25
:10583000AAF10100216B01EB800828F0070808F0AD
:10584000070008B9012000E0002028B940F22B32FF
:105850001BA122A0FCF79CFE002507E0795D04F166
:1058600034004155785D00B902E06D1C102DF5D370
:1058700000BF002143200155202E00D31F26E662E1
:1058800066640020A064201D02F0C9FD04F1180028
:1058900002F0C5FD2461C6F12000A0616462002011
:1058A000E06484F8500049464046039A00F0D6FB75
:1058B0002060BBF1000F01D0CBF80040BDE8FF9F96
:1058C0002E2E5C2E2E5C4672656552544F535C73CF
:1058D00072635C7461736B732E6300004572726F48
:1058E000723A25732C25640D0A0000002DE9F0475B
:1058F00006460D4617469846DDE908940DB101208D
:1059000000E0002028B94FF4C67209A10FA0FCF7EF
:105910003FFE5CB1FFF73CFE2660A561E761C4F87D
:105920002080C4F82490201D02F079FDBDE8F087A6
:105930002E2E5C2E2E5C4672656552544F535C735E
:1059400072635C74696D6572732E63004572726F69
:10595000723A25732C25640D0A00000010B500244E
:1059600007E004EB84010F4A02EB810002F04AFDDC
:10597000641C202CF5D30C4802F044FD0B4802F0C7
:1059800041FD0B4802F03EFD0A4802F03BFD0A488B
:1059900002F038FD044809490860044808490860D5
:1059A00010BD0000A80A0020280D00203C0D00209A
:1059B000500D0020640D0020780D002040010020D3
:1059C0004401002010B50146164800E00068036855
:1059D0008B42FBD30246436813448B4204D1436895
:1059E0004C682344436001460A464B6813440468EC
:1059F000A34211D10C4C03682468A34208D04B6821
:105A00000468646823444B6003681B680B6005E00E
:105A1000054B1B680B6001E003680B60884200D0F7
:105A2000016010BD8C010020940100202DE9F0419F
:105A300004460D4616461F464FF000086560246177
:105A4000B5420CD8F01BA169884202D34FF001087F
:105A500011E0211D0948006802F0E4FC0BE0BE42A1
:105A600004D2BD4202D34FF0010804E0211D0448D6
:105A7000006802F0D7FC4046BDE8F0817C010020C0
:105A80007801002070B5054602F0F2FCA86B08B959
:105A9000012400E0002402F02DFD204670BD70B509
:105AA000054602F0E5FCA86BE96B884201D10124B0
:105AB00000E0002402F01EFD204670BDF8B505464A
:105AC0000F4613480068C068C468201D02F086FCB9
:105AD000E069012818D1A06941192B463A462046B1
:105AE000FFF7A4FF80B1002003462A46014600903C
:105AF000204603F0D9FF06462EB94FF4027205A1E5
:105B00000BA0FCF745FD00BF2046616A8847F8BD41
:105B1000780100202E2E5C2E2E5C46726565525454
:105B20004F535C7372635C74696D6572732E6300AE
:105B30004572726F723A25732C25640D0A000000BD
:105B400070B586B060E0039800285DDB059C606955
:105B500008B9012000E0002010B9201D02F03EFC31
:105B600002A800F0C9F8054603980A284AD2DFE8DF
:105B700000F00905072C2E4506082D2F00BF00BF99
:105B800000BF00BF0498A269811803462A46204638
:105B9000FFF74CFFC0B12046616A8847E0690128E1
:105BA00012D1002000900498A169421800231946E0
:105BB000204603F079FF06462EB940F2213218A1A3
:105BC0001EA0FCF7E5FC00BF1DE000BF1BE000BF0E
:105BD0000498A061A06908B1012000E0002028B964
:105BE0004FF44E720EA115A0FCF7D2FCA06941192A
:105BF0002B462A462046FFF719FF04E0204602F014
:105C0000AFFC00E000BF00BF00231A4603A90F4805
:105C1000006803F0A7F9002895D106B070BD000018
:105C20002E2E5C2E2E5C4672656552544F535C736B
:105C300072635C74696D6572732E63004572726F76
:105C4000723A25732C25640D0A00000080010020A3
:105C5000F8B505460C4602F083FF684600F04CF8A4
:105C60000646009820BB44B9B54206D803F034FE7E
:105C700031462846FFF722FF1CE03CB10E48006881
:105C8000006808B9012000E000200446A91B224654
:105C90000A48006802F034FD03F01EFE50B94FF0D0
:105CA000805007490860BFF34F8FBFF36F8F01E04B
:105CB00003F012FEF8BD00007C01002080010020EE
:105CC00004ED00E00A490968096809B9012100E00A
:105CD000002121B14FF0FF31064A116006E004496E
:105CE0000968C968C868034A4168116070470000C4
:105CF000400100206C01002070B5044603F064FCF4
:105D0000054607480068854204D200F00BF80120E0
:105D1000206001E00020206001480560284670BD39
:105D2000880100202DE9F8432DE021480068C06873
:105D300005681F480068C068C468201D02F04EFB5B
:105D40002046616A8847E06901281CD1A06946198C
:105D5000AE4207D966602461211D1548006802F033
:105D600061FB10E0002003462A46014600902046D1
:105D700003F09AFE07462FB940F292320DA114A00B
:105D8000FCF706FC00BF0A480068006808B901205B
:105D900000E000200028C8D00548D0F80080104856
:105DA0000068034908600E48C0F80080BDE8F88329
:105DB000780100202E2E5C2E2E5C467265655254B2
:105DC0004F535C7372635C74696D6572732E63000C
:105DD0004572726F723A25732C25640D0A0000001B
:105DE0007C0100200B480068401C08B9012000E03D
:105DF000002020B9F42208A111A0FCF7C9FB00BFC4
:105E0000502080F31188BFF34F8FBFF36F8F00BF17
:105E100000BFFEE7A40100202E2E5C2E2E5C4672F1
:105E2000656552544F535C706F72745C52564453A4
:105E30005C41524D5F434D335C706F72742E630052
:105E40004572726F723A25732C25640D0A000000AA
:105E500008B500BF6846FFF75BFC04462046009982
:105E6000FFF7F6FEFFF76CFEF4E770B5044602F0AC
:105E7000FFFA94F9455010E0606A08B9012000E08B
:105E8000002038B904F1240003F0C8FC18B102F076
:105E900025FD00E003E0681E45B2002DECDC00BFEC
:105EA000FF2084F8450002F025FB02F0E1FA94F9A6
:105EB000445010E0206908B9012000E0002048B9F2
:105EC00004F1100003F0AAFC08B102F007FD681EFF
:105ED00045B200E001E0002DECDC00BFFF2084F8BB
:105EE000440002F007FB70BD2DE9F04104464FF07D
:105EF000000802F035FE3E48006808B9FFF71CFCB8
:105F00003C480068204000285FD1A4B1083404F068
:105F1000070080B104F00700C0F10800044404F059
:105F2000070008B9012000E0002020B9BF2232A1FB
:105F30003BA0FCF72DFB002C47D03D480068844275
:105F400043D83C4E3046056801E02E462D6868680F
:105F5000A04202D228680028F7D12548006885426F
:105F600033D0306800F10808286830606868001B8A
:105F7000102813D92F1907F0070008B9012000E0F5
:105F8000002020B9EC221CA125A0FCF701FB6868C9
:105F9000001B78606C603846FFF714FD2449686880
:105FA0000968081A224908600846006822490968F9
:105FB000884203D21E4800681F4908600D4968687E
:105FC0000968084368600020286003F085FC08F039
:105FD000070008B9012000E0002028B94FF49672AC
:105FE00005A10FA0FCF7D4FA4046BDE8F0810000FF
:105FF00094010020A00100202E2E5C2E2E5C467203
:10600000656552544F535C706F72745C4D656D4D95
:10601000616E675C686561705F342E63000000002C
:106020004572726F723A25732C25640D0A000000C8
:10603000980100208C0100209C0100200648006887
:1060400030B10549096801F14800896C491C0160BB
:1060500001480068704700003C010020001F4FF01D
:1060600080730360001F21F001030360001F034BD6
:10607000036014380260203870470000E55D0008B6
:1060800000487047400A00202DE9F04794B00446CC
:106090004FF00009CA4628220AA9206BFEF7A4F88F
:1060A00006210AA8FEF7E2FE20701098A060A06802
:1060B000401C30B1A068B0F5006F02D8A06820285D
:1060C00019D22820A060207805280ED00520207045
:1060D00035A240F21B2140A0236BFDF7BFFF052333
:1060E00006220AA9206B02F015FE00206070022033
:1060F00014B0BDE8F087A068B0F5777F0ED9A0682E
:10610000B0F5006F0AD23C483CA33DA240F22221E8
:10611000009031A0FDF7A2FF00BFFEE7A068A0F14C
:1061200020060025002716E005F12000B04201D22C
:10613000202700E0771BF91C21F00302216B20319E
:10614000481902A9FEF750F83A4602A94846FDF759
:106150004FFD81463D44B542E6D31198484504D0F1
:10616000002060704FF0020A1BE001206070206B7D
:1061700000F128089DF84800C01C20F0030204F13B
:1061800010014046FEF730F89DF84800C01C20F092
:10619000030000EB080161631398E0609DF848007C
:1061A000A0705046A4E700004572726F723A205406
:1061B000686520454E562040307825303858206C90
:1061C000656E6774682068617320616E2065727205
:1061D0006F722E0A000000002E2E5C2E2E5C55736E
:1061E00065725C6561737964625C7372635C656639
:1061F0005F656E762E630000659B0008300000002E
:106200002825732920686173206173736572742077
:106210006661696C65642061742025732E0A000034
:1062200070B5002406A0FDF739FE05460022114690
:106230002846FAF719F884B2FFF722FF848270BD6E
:106240006B65795F656E5F7461626C65000000006C
:1062500070B509A0FDF722FE05462846FAF73DF87D
:10626000C4B2FFF70DFF8472FFF70AFF847A21465C
:1062700003A0FCF78DF970BD6B65795F73000000BA
:10628000E99481E5AE9AE697B6E997B43A25640DAC
:106290000A0000002DE9F04198B005460C4617466B
:1062A0004FF00008C5F3090050B14F484FA355A265
:1062B00040F2492100905BA0FDF7D0FE00BFFEE751
:1062C00054B949485FA34FA240F24A21009055A01B
:1062D000FDF7C4FE00BFFEE724220FA92846FDF704
:1062E00083FF65601598A0605849A068884207D070
:1062F00000202070401EE060072018B0BDE8F0814B
:10630000012020701698E06004210FA8FEF7AEFD72
:106310006070042112A8FEF7A9FDA070002F60D0C4
:10632000002020616068243060616078012803D11A
:106330004FF47770206154E06078022851D104F165
:1063400014012846FEF77AFD38B161686069401A89
:10635000C0F5806020614046CFE74FF47770206140
:106360004FF0FF300D901EE001A8FFF78DFE9DF865
:10637000050080B99DF8040001280CD09DF80400A8
:10638000052808D032A00D99FDF794FE0020206169
:106390004FF002080FE060690399084460612069CA
:1063A0000399401A206101A92046FEF7F1FC0D90E7
:1063B000401C0028D8D100BF626802F58061606986
:1063C000FDF722F906466069B04205D06661606853
:1063D000301AC0F5806020616169606801F044FE98
:1063E00000BF404689E700006E9B0008616464724C
:1063F000202520534543544F525F53495A45203D71
:106400003D20300028257329206861732061737353
:10641000657274206661696C6564206174202573FF
:106420002E0A00002E2E5C2E2E5C557365725C6564
:1064300061737964625C7372635C65665F656E76D6
:106440002E630000736563746F720000454634303C
:106450004572726F723A2054686520454E56202866
:106460004030782530385829204352433332206356
:106470006865636B206661696C6564210A000000D1
:10648000F8B506460C46154654B90C480CA310A2A4
:1064900040F22711009016A0FDF7E0FD00BFFEE7D7
:1064A000681E072101EB4010C20821463046FDF767
:1064B0009BFE29462046FEF7D9FCF8BD599B0008F3
:1064C0007374617475735F7461626C6500000000C1
:1064D00028257329206861732061737365727420A5
:1064E0006661696C65642061742025732E0A000062
:1064F0002E2E5C2E2E5C557365725C65617379641B
:10650000625C7372635C65665F656E762E63000025
:106510002DE9F04704460D4616461F46DDE9088979
:106520004FF0FF3060601AE0002221465046FFF72E
:10653000B1FE15B16078A84211D1B9F1000F04D0B5
:106540004A4621465046FFF7A5FEB8F1000F06D097
:106550003A4631462046C04708B1BDE8F08720469C
:10656000FEF74CFC8246401C0028DDD100BFF4E75A
:1065700030B503460C461546187830B158780128D6
:1065800003D12068401C206007E0187828B15878B3
:10659000022802D12868401C2860002030BD00007D
:1065A0002DE9F04706460C4617460025A84634B9A3
:1065B000012200213046FDF783F9054632E03046DE
:1065C000F9F72EFE81463A4649461748FEF726FF60
:1065D000401C10B90620BDE8F08714493046FDF78D
:1065E000C6FE8046B8F1000F05D000220F493046A4
:1065F000FDF766F9054635B93B46224631460A485D
:10660000FDF736F80546B8F1000F06D02DB9012286
:1066100006493046FDF754F905460548007808B1AB
:10662000FEF7A6F92846D6E710370020D836002016
:10663000E90100202DE9F04105460E4614464FF0D1
:10664000FF37701E072202EB4010C108FF222846C8
:10665000F9F7C8FD1CB1601E87000020E8553846D8
:10666000BDE8F0810146002009E0074A52F82020E9
:106670001AB9054A42F820107047421C10B20A2885
:10668000F3DB00BFF8E70000A837002010B5044690
:106690000121204600F075F810BD000010B5044639
:1066A000226891682069F9F7C2FD60B994F860002A
:1066B00020F00100401C84F8600008480168204672
:1066C00001F01CFB04E00548416B204601F016FB7D
:1066D0000020A0810021E18110BD0000EC0100201C
:1066E0000246087858B1487800F00F00082806D014
:1066F000106878B1087813681B78184050B192F888
:10670000600000F0010018B94878C0F3001008B12B
:10671000002070474FF0FF30FBE7000010B500F09D
:1067200017FB044624B10348816B204601F0E6FACA
:1067300010BD0000EC01002070B50446A189E0897D
:10674000081A05B205E02021204601F027FA681E4C
:1067500005B2002DF7DC217B204600F07FF870BDEC
:1067600010B500F0F5FA044614B1204600F054FDCF
:1067700010BD10B504464FF0FF31204600F001F87F
:1067800010BD2DE9F04104460D46681C08B90120F2
:1067900000E000200746E08908B9012D05D0E08916
:1067A000A189884203D1681C08B9BDE8F081E0895D
:1067B000A189884210D1012D0ED1E089401EE081CF
:1067C000A089401EA0810021A28920698154012155
:1067D000204600F043F83FE038460AE0E1890144F2
:1067E0002269525CE1890144491E23695A54411CC3
:1067F00008B2A289E189511A8142EFDCA089401ECA
:10680000A08137B9E089401EE0810821204601F0CF
:10681000C5F90021A28920698154E08906B206E009
:106820002069815D204601F0B9F9701C06B2A0898B
:10683000B042F5DC2021204601F0B0F9A189E089C1
:10684000081A401C06B205E00821204601F0A6F90E
:10685000701E06B2002EF7DC00BFA6E770B5054635
:106860000C4603E004A1284601F048FA201EA4F1DA
:106870000101CCB2F6D170BD0820080010B5044665
:106880004FF0FF31204600F047FB10BD10B5044625
:10689000204600F005F80121204601F0B5F910BDB1
:1068A00070B50446A08900B970BD0021A289206995
:1068B000815494F8600000F0010010B3204600F00D
:1068C0008CFB204600F09CFD0021E181A181E08E3F
:1068D00000B9E9E70DA1204601F010FA0023204697
:1068E000A26D616900F035FE054625B129462046B6
:1068F00000F0D6FD04E006488169204601F0FEF96B
:1069000002E02046FFF7CAFE00BFCDE70D0A0000F7
:10691000EC01002010B50246114600200B78302B08
:1069200007D14B78782B02D04B78582B01D103201C
:106930000EE00B78302B07D14B78622B02D04B78CE
:10694000422B01D1012003E00B78302B00D1022033
:1069500006E00B782E2B03D14B780BB1042003E01B
:1069600011F8014B002CF4D100BF10BD0246137882
:10697000272B01D1531C00E01346194600200B7849
:106980005C2B1AD14B786E2B0ED004DC302B0FD041
:10699000622B0FD104E0722B04D0742B0AD105E0D6
:1069A000082009E00D2007E00A2005E0092003E0A7
:1069B000002001E0487800BF00E0087870472DE92A
:1069C000F04F85B005464FF000094FF00A0A2C46FB
:1069D000CB460126002700200490804628782D28E9
:1069E00000D1B61E711C09B9012100E0002148192F
:1069F000FFF790FF8146B9F1010F0FD0B9F1020FF7
:106A000007D0B9F1030F0DD14FF0100A4FF0020B70
:106A100009E04FF0080A4FF0010B04E04FF0020AC2
:106A2000D34600E000BF00BF05EB0B01701C08B9A6
:106A3000012000E000200C1811E020782E2803D15E
:106A40004FF00108641C0AE0207800F026F907FBEB
:106A50000A0708EB88004FEA4008641C00BF207852
:106A60000028EAD1B9F1040F1AD1B8F1000F17D0FC
:106A70003046F9F790FD03904046F9F795FD0190F7
:106A80003846F9F791FD00900199F9F765FC0290FD
:106A90000399F9F72FFC0490049805B0BDE8F08F36
:106AA00007FB06F0F9E72DE9F04107460C461646CC
:106AB0001D4626B1207824282FD1607868B320782D
:106AC000272808D1607830B12046FFF74FFF2860B3
:106AD0000020BDE8F08120782D2805D020783028CE
:106AE00008DB2078392805DC2046FFF768FF28609E
:106AF0000020EEE72078242807D1607828B12A46C4
:106B00002146384600F031F8E3E7207828B12046E6
:106B100000F006F828600020DBE74FF0FF30D8E7F0
:106B200070B50446254600262078222802D1601C34
:106B30000446054613E028785C2805D12846FFF76F
:106B400015FFA0556D1C07E02878222802D10020EF
:106B5000A05501E02878A0556D1C701C86B22878DD
:106B60000028E8D1A055204670BD2DE9F04104462B
:106B70000D4616460023691C2046A26D00F0E9FC74
:106B800007463FB13946204600F0FCF8306000204F
:106B9000BDE8F0814FF0FF30FAE72DE9F0478CB007
:106BA00080460C4615461E464FF0000A202104A8D8
:106BB000F9F71FFBA07800F00F01681E814203DD8A
:106BC000A07800F00F0000E0681E07464FF00009B3
:106BD00012E004A800EB890309F1010056F8201027
:106BE00000224046FFF75FFF20B14FF0FF300CB0AE
:106BF000BDE8F08709F10109681E4845E9DC082F66
:106C000045D2DFE807F004080E151C232C37A068D6
:106C1000804782463EE0D4F808900498C8478246F0
:106C200038E0D4F80890DDE90401C847824631E035
:106C3000D4F8089004A807C8C84782462AE0D4F8C8
:106C4000089004A80FC8C847824623E0D4F80890EB
:106C50000898009004A80FC8C84782461AE0D4F8E4
:106C60000890DDE90801CDE9000104A80FC8C84774
:106C700082460FE0D4F80890DDE908120A98CDE9C1
:106C80000012029004A80FC8C847824602E04FF0E5
:106C9000FF3A00BF00BF5046A9E70146302905DB97
:106CA000392903DCA1F13000C0B27047612905DB4E
:106CB000662903DCA1F15700C0B2F6E7412905DBE4
:106CC000462903DCA1F13700C0B2EEE70020ECE773
:106CD0000146487800F00F00012801DCC8687047C1
:106CE000487800F00F00072801DCC868F7E748780B
:106CF00000F00F00082801DCC868F0E7C868EEE77C
:106D000010B50446002004E03021104A1154411C03
:106D1000C8B20928F8DB607800F00F00012801DC18
:106D2000606810BD607800F00F00072801DC606823
:106D3000F7E7607800F00F00082801DC6068F0E7F2
:106D40000249606800F0F5FE0048EAE7D03700200D
:106D5000002111E00A4850F8210058B1084850F8C5
:106D6000210090F86000C0F3400018B1044850F8CA
:106D700021007047481C01B20A29EBDB0020F8E72C
:106D8000A83700202DE9F04107460C460026607820
:106D900000F00F00801E06281BD2DFE800F003067B
:106DA0000A0D0E10A068066814E0A068B0F9006033
:106DB00010E0A06806780DE000BFA6680AE0A068B1
:106DC00045681DB1A1680868A84700E00020064694
:106DD00000E000BF00BF3046BDE8F0812DE9F0477C
:106DE00004468846B8F1000F01D1BDE8F08720467F
:106DF000E16E884720688068A0B121688868F9F74B
:106E00000FFA78B102F0E0FB60B102F0DDFB6168DF
:106E1000401A3F49884205D994F8600020F00100EB
:106E200084F8600018274FF00009208F00F47F409D
:106E300018B100276FF0FF090EE0A06B00F47F008F
:106E400018B10827DFF8CC9006E0A06B00F07F4077
:106E500010B110274FF07F49A66D00253EE006EBEC
:106E60000510407800F00F00092835D106EB051118
:106E70002046FFF735FC70BB06EB0510406800EAC2
:106E80000900A16B884227D106EB05104068FF215D
:106E9000B940084008FA07F188421DD108FA07F105
:106EA000A06B0843A0634FF0000847B106EB051044
:106EB0004068A7F10801FF228A40104058B906EB4C
:106EC0000510806820B106EB0510816820468847D0
:106ED0000021A16306E0FFE7681C05B25C20005BAF
:106EE000A842BCDC00BFB8F1000F05D00021A163AF
:106EF0004146204600F076FA02F066FB10B102F03F
:106F000063FB60602046216F884700BF6DE700008B
:106F1000E09304000000FFFF70B504460D46002D0D
:106F200025DDB4F954105420005B401E02B25420F9
:106F300002535020025B5220005B824202DD50204F
:106F4000005B01E05220005B404281421DDC50208A
:106F5000015B5220005B814202DD5020005B01E0BA
:106F60005220005B404201B2542001530DE0002D3D
:106F70000ADA5420005B401C01B25420015300295E
:106F800003DD0021015370BDFDE72046FFF7D4FB70
:106F90005420005B18B90021A181E1811BE052203F
:106FA000005B401DB4F954100844052190FBF1F238
:106FB00001FB120104F13C0050F8216031462069C8
:106FC00000F0ACFCA08100B9DDE7A189E181204699
:106FD000216900F093FE00BFD5E710B504460021FB
:106FE000542001535020005B002810DD5222125B18
:106FF00021690AB9052201E05222125B521E04F1F6
:107000003C0353F82200F9F712F900B910BD5222DF
:10701000135B04F13C0252F82300216900F07EFC6E
:1070200028B15220005B401C81B2522001535020F5
:10703000005B401C81B250200153052901DD052170
:1070400001535220005B052802DB0021522001532E
:1070500000BFDBE72DE9F04104460D46164600204F
:10706000A0810021E181206094F8600020F00100FF
:10707000401C84F860002561062096FBF0F0A08695
:10708000542001535020015352200153002009E0A5
:10709000A28E411C02FB015204F13C0141F8202068
:1070A000411C08B20528F3DB0E48A0650E480D49C7
:1070B000401AC0F30F115C2001532046FFF7D2FAAB
:1070C00000230AA12046A26D00F043FA0746394684
:1070D000204600F07BFA0121204600F095FDBDE836
:1070E000F081000064A60008C4A700087A696974EA
:1070F0000000000070B504460D46A189A08E401E18
:1071000081420DDB38484168204600F0F7FD01213F
:10711000204600F079FD2046216900F0EFFD70BDAA
:10712000E089A189884218D1A189481CA0812069E1
:1071300045540021A28920698154E089401CE081E6
:1071400094F8600000F0010008B1284600E02A2011
:107150000146204600F022FD44E0E089A1898842F2
:1071600040DAA289E189511A08B20AE0E1890144B2
:10717000491E2269525CE189014423695A54411E27
:1071800008B20028F2DCE189481CE08120694554FE
:107190000021A089401C80B22269A0811154E0899D
:1071A000401E06B20EE094F8600000F0010010B13D
:1071B0002069805D00E02A200146204600F0EEFCB8
:1071C000701C06B2A089B042EDDCA189E089081AE2
:1071D00006B205E00821204600F0E0FC701E06B271
:1071E000002EF7DC00BF9AE7EC01002010B5044642
:1071F000E089002806DD0821204600F0CFFCE08968
:10720000401EE08110BD10B50446204600F092F803
:10721000204600F001F810BD70B50546AE6D10486F
:107220008168284600F06AFD002413E006EB041094
:10723000407800F00F0001280ADC06EB0411284614
:10724000FFF74EFA20B906EB0411284600F00AF8C1
:10725000601C04B25C20405BA042E7DC70BD000013
:10726000EC0100202DE9F04106460C462046FFF7D0
:1072700047FD07463946304600F040FDC0F1140096
:1072800005B2002D01DD284600E00220054600BFC2
:1072900024A0FBF77DF9681E00B2051EF8D16078C6
:1072A00000F00F00012805DC1F48016C304600F09B
:1072B00025FD25E0607800F00F00072805DC1A485E
:1072C000416C304600F01AFD1AE0607800F00F00C3
:1072D000082805DC1448816C304600F00FFD0FE0F3
:1072E000607800F00F00092805DC0F48C16C3046BB
:1072F00000F004FD04E00C48016D304600F0FEFC97
:107300000AA1304600F0FAFC2046FFF7E1FC0746F0
:107310003946304600F04AFC05A1304600F0EEFC4C
:10732000BDE8F08120000000EC01002020200000DA
:107330000D0A000070B50646B56D13480169304668
:1073400000F0DCFC00241AE005EB0410407800F0AB
:107350000F00072811DD05EB0410407800F00F0046
:1073600008280ADC05EB04113046FFF7B9F920B90B
:1073700005EB04113046FFF775FF601C04B25C207A
:10738000805BA042E0DC70BDEC01002070B50646D9
:10739000B56D1348C168304600F0B0FC00241AE017
:1073A00005EB0410407800F00F00012811DD05EB1B
:1073B0000410407800F00F0007280ADC05EB0411E8
:1073C0003046FFF78DF920B905EB04113046FFF781
:1073D00049FF601C04B25C20805BA042E0DC70BD11
:1073E000EC01002070B504460D4694F8600020F0D2
:1073F000040084F8600029462046FFF77BFE70BD3C
:1074000018B5044608200090A189202304F1140235
:10741000206900F0E1F9E08618BD70B5044600254A
:107420002BE004F1140050F82500007822280CD13C
:10743000002104F1140050F82500017004F114003B
:1074400050F82510491C40F8251004F1140151F89A
:107450002500F8F7E5FE86B204F1140050F8251077
:10746000701E085C222806D1002104F1140050F897
:107470002520701E1154681C85B2E08EA842D0DC15
:1074800070BD10B50446E089A189884207DAE28917
:10749000501CE0812069815C204600F07FFB10BD1C
:1074A0002DE9F04104460D46002694F8600020F0D6
:1074B0000200801C84F86000687800F00F0088B932
:1074C0002046FFF7AAFFAF68E08E04F11401B84729
:1074D00006466878C0F3401018B93146204600F0DF
:1074E000C7FB2DE0687800F00F00012810D1E28E74
:1074F00004F1140329462046FFF74FFB064668783F
:10750000C0F34010E0B93146204600F0B1FB17E06F
:10751000687800F00F00022809DB687800F00F009F
:10752000072804DC2946204600F002F908E06878C4
:1075300000F00F00082803D12946204600F046F845
:1075400094F8600020F0020084F860003046BDE846
:10755000F0812DE9F0470646884614461F465C2018
:10756000805BB16D611AA0EB11101FFA80F9002544
:1075700028E004EB0510407800F00F00092805D042
:1075800004EB05113046FFF7ABF800B118E004EB4F
:107590000510FFF7B5FB824647B951464046F8F75C
:1075A00046FE60B904EB0510BDE8F0873A46514647
:1075B0004046F8F74AFE10B904EB0510F4E700BFA7
:1075C000681C85B24D45D4DB0020EDE770B504465C
:1075D0000D462560A86858B1A868F8F721FE38B1B3
:1075E000E08E022806DBA169A868F8F720FE08B93A
:1075F000012000E0002094F8601060F3000184F89E
:1076000060100848816B204600F078FB94F8600019
:1076100000F0010020B103480168204600F06EFB35
:1076200070BD0000EC0100202DE9F04106460F4638
:10763000FFF78EFB054615B90020BDE8F081002359
:1076400031462846AA6DFFF784FF044634B9114835
:10765000816A284600F052FB0020EEE7607800F0D7
:107660000F00022804DB607800F00F0007280ADD15
:107670003146284600F042FB0648416A284600F0A1
:107680003DFB0020D9E73A462146284600F004F8A1
:10769000D3E70000EC0100202DE9F04106460C463E
:1076A00015466078C0F3801028B12048016A304642
:1076B00000F024FB34E0607800F00F00801E062804
:1076C0002CD2DFE800F003060A0D1218A06805604E
:1076D00025E029B2A068018021E0A06805701EE0C5
:1076E0002946A06800F01AF919E01048C16930462F
:1076F00000F004FB13E0A068806870B1A068006827
:1077000030B1A0688768A16808682946B84704E0D6
:10771000A06887682846B84700BF00E000BF00BFE8
:107720002146304600F004F8BDE8F081EC0100206D
:10773000FEB505460C4622A207CA8DE80700214681
:107740002846FFF71FFB07462846616800F0D6FA77
:107750001EA1284600F0D2FA607800F00F0005283C
:107760000CD11BA1284600F0C9FA3946284600F082
:10777000C5FA17A1284600F0C1FA19E06946384653
:1077800000F0ACF9C0F10B006946461831462846B6
:1077900000F0B4FA002004E030210DF80010411C84
:1077A00008B20B28F8DB6946284600F0A7FA00BFAC
:1077B00000BF08A1284600F0A1FA3846FEBD00002F
:1077C000303030303030303030303000203D20002C
:1077D000220000000D0A00002DE9FF4F04468C46F0
:1077E00015460D9F4FF00108002000900190029077
:1077F00003900021002600BF04E0002245F820206D
:10780000421C10B2B842F8DB002068E011BB225CD9
:107810009A420DD0B8F1010F0AD1BE4208DA04EB4A
:10782000000A3246761C45F822A04FF0000811E00D
:10783000225C9A4202D0225C202A0BD1B8F1000FC0
:1078400008D100222254421CA25C202A01D04FF011
:10785000010842E0002234E0002918DD14F800900D
:10786000DFF888A00AEB420A9AF801A0D1450ED1B0
:10787000A1F101091DF80990DFF870A01AF812A013
:10788000D14504D1A1F1010909F0FF011BE014F871
:107890000090DFF858A01AF812A0D1450DD1DFF8FA
:1078A0004C9019F812B0894601F1010A0AF0FF0163
:1078B0000DF809B001F00F0105E002F1010909F02E
:1078C000FF02002AC8D000BF225C5C2A04D1421CFF
:1078D000A25C0AB1421C90B200BF421C90B260454B
:1078E00094DB304604B0BDE8F08F00004002002079
:1078F00030B502460B460020002108E0545C5D5C78
:10790000AC4200D008E0441CA0B24C1CA1B2545CB4
:1079100014B15C5C002CF1D100BF30BD02460020E8
:1079200003E00B5C1354431C98B20B5C002BF8D1A2
:10793000135470472DE9F84F0446B4F834A04FF0C3
:1079400000080025A08938B92046FFF75CFC01211A
:10795000204600F059F970E0A08900286DDD002173
:10796000A28920698154A66D002737E006EB071134
:107970002046FEF7B5FE78BB06EB0710FFF7C0F90F
:10798000834659462069FFF7B3FFA189884223D176
:10799000F5B1012D03D145A1204600F0AFF906EB6A
:1079A00008112046FFF75EFC06EB0710FFF7A8F969
:1079B000834606EB0810FFF7A3F959460090FFF73E
:1079C00097FF8146CA4501DD484600E050468246A1
:1079D0001FFA87F8681C85B2781C07B25C20005B30
:1079E000B842C3DC0DB9BDE8F88F012D02D12046A5
:1079F000FEF7A2FE4DB106EB0810FFF781F907462E
:107A000039462069FFF78AFFA081012D0ADD06EBC8
:107A100008112046FFF726FC0121204600F0F4F86B
:107A2000A4F80CA00021A28920698154A189E181D8
:107A30002046216900F062F900BF01F0C5FD58B38E
:107A4000012D2AD194F86000C0F3800028B301F022
:107A5000BBFD6168401AC8281FD22046FEF76CFEA5
:107A6000A18908B206E021690A5C0B46411D5A54FF
:107A7000411E08B20028F6DA0DA12069FFF74EFF7B
:107A8000202120690171A089401DA081A189E18187
:107A90002046216900F032F906E094F8600020F0F9
:107AA0000400001D84F8600000BF9CE70D0A000080
:107AB00068656C700000000008B505462C460CE0B7
:107AC000606E50B101216846626E9047012804D172
:107AD0009DF800102046FFF781F9F1E730B5024626
:107AE0000B241346002A00DA53420020C8720DE02E
:107AF0000A2093FBF0F500FB15303030C5B2601E54
:107B0000C0B204460D540A2093FBF0F3002BEFD1D2
:107B1000002A04DA2D25601EC0B204460D5422B995
:107B20003025601EC0B204460D54C4F10B0040B2B3
:107B300030BD30B502460B460824002018720EE016
:107B400002F00F01092902DD01F1570001E001F106
:107B50003000C5B2601EC0B204461D541209002A8E
:107B6000EED1C4F1080040B230BD10B50446012189
:107B70002046FFF7D1F910BD10B5FFF7E9F804462C
:107B800014B12046FFF7D6FB10BD10B5FFF7E0F8A3
:107B9000044614B12046FFF7F9FB10BD13B50446A7
:107BA000012101A8A26E90471CBD00002DE9F04103
:107BB00004460F4600253E46A06E10B90020BDE8E1
:107BC000F08102E0761C681C85B2307828B13078EC
:107BD0000D2802D030780A28F4D1242D08DD242184
:107BE0003846A26E9047032106A0A26E904703E09C
:107BF00029463846A26E9047242D01DD2420DEE779
:107C00002720DCE72E2E2E0070B504460D4694F892
:107C1000600000F00100D8B11DB110A1204600F0B5
:107C20006DF820684168204600F068F80CA12046F5
:107C300000F064F8A06808B1A06800E009A001465F
:107C4000204600F05BF808A1204600F057F804E059
:107C50000648016B204600F051F870BD0D0A000087
:107C60003A0000002F00000024200000EC0100205A
:107C7000FEB505460C4618A2D2E900109268CDE97F
:107C80000102009117A1284600F038F86946204605
:107C9000FFF724FFC0F10B0069464618314628461D
:107CA00000F02CF812A1284600F028F8002004E08B
:107CB00030210DF80010411C08B20B28F8DB694692
:107CC0002046FFF736FF6946284600F017F80AA15C
:107CD000284600F013F8FEBD303030303030303000
:107CE0003030300052657475726E3A20000000002A
:107CF0002C203078000000000D0A00002DE9F04132
:107D000004460D4600262F46A06E10B90020BDE89F
:107D1000F08101E0701C86B217F8011B0029F9D12F
:107D200031462846A26E904780B2F0E77CB5FFF757
:107D30000FF80546002000900190FEF7A1F94FF6DC
:107D4000FF718182FEF79CF9848A234615A20621E1
:107D50006846FAF72DFC694614A0FCF791FA17A0C3
:107D6000FAF716FCFEF78CF90A218172FEF788F902
:107D7000847A23461FA206216846FAF719FC694651
:107D80001DA0FCF77DFA1EA0FAF702FCFCF776FABC
:107D900018B925A0FAF7FCFB02E02FA0FAF7F8FBD0
:107DA0007CBD000030782558000000006B65795FCD
:107DB000656E5F7461626C6500000000E68C89E9A5
:107DC00094AEE4BDBFE883BDE8A1A8E5B7B2E8AED4
:107DD000BEE7BDAEE4B8BA3A203078464646462003
:107DE00028E585A8E983A8E4BDBFE883BD290D0A7D
:107DF00000000000256400006B65795F73000000DF
:107E0000E68C89E994AEE4BC91E79CA0E697B6E9DC
:107E100097B4E5B7B2E8AEBEE7BDAEE4B8BA3A2073
:107E2000313020730D0A0000E58F82E695B0E5B78A
:107E3000B2E4BF9DE5AD98E887B320466C617368F6
:107E4000EFBC8CE9878DE590AFE5908EE7949FE6D7
:107E500095880D0A00000000E8ADA6E5918AEFBC08
:107E60009AE58F82E695B0E4BF9DE5AD98E887B3CB
:107E700020466C61736820E5A4B1E8B4A50D0A0042
:107E800010B5FEF7FDF80078012805D1FEF7F8F8E7
:107E9000841D8079401C2070FEF7F2F88479FEF78B
:107EA000EFF8807A844214DBFEF7EAF80021417093
:107EB000FEF7E6F800210170FEF7E2F8002181717B
:107EC0004FF480710348F9F754FC034841680020DF
:107ED000884710BD000C01402C0000202DE9F04126
:107EE00004460D4616461F464FF0000806E0A04720
:107EF0003846A84708F1010000F0FF08B045F6DB5E
:107F0000BDE8F0812DE9F05F81468A4615461026CE
:107F10001027524649460020FBF76AFE4FEA1048F8
:107F20004FF6FF7B00244BE0681CB0B3354830F8B7
:107F30003400404505D1334800EBC4004560BDE83E
:107F4000F09F304800EBC4004068401C18B9102E68
:107F500001D1264633E02B4800EBC4004068401CAA
:107F600068B3284800EBC4004088002808DD254895
:107F700000EBC4004088401E224901EBC401488048
:107F8000204800EBC4004088584518DA27461D48B1
:107F900000EBC400B0F802B011E0FFE7194830F878
:107FA000340040450BD14FF0FF30164901EBC401BE
:107FB00048600020134901EBC4014880BFE7641CFE
:107FC000102CB1D3102E0CD20E4800EBC600456029
:107FD0000C4820F8368000200A4901EBC601488091
:107FE0000DE0102F0BD2074800EBC7004560054895
:107FF00020F837800020034901EBC701488000BF0B
:108000009DE70000B4350020FEB504460E46154637
:1080100000276078012807D102230422694660689E
:1080200000F078FE07461DE0607802281AD120692A
:10803000482803D32069801B482810D20323042238
:108040006946606800F066FE0746626802F5806176
:10805000104600F009F82DB10120287002E00DB1A2
:10806000002028703846FEBD30B5024604230020AB
:1080700026E0914218D902F58064A14214D2164C30
:1080800054F83040944206D1134C44F8302004EBAD
:10809000C004616030BD104C54F83040641C74B9A9
:1080A000042B0CD103460AE00B4C54F830409442A8
:1080B00005D14FF0FF34084D45F83040EAE7401C49
:1080C0000428D6D3042B05D2034C44F8332004EB08
:1080D000C304616000BFDDE7343600201CB5012019
:1080E00000F0F0FE104908601048114988661148F8
:1080F00048661148C866114808674FF40072104975
:108100000B48FEF7A7FF00200521094B4FF48072B2
:10811000CDE900100BA10D4801F016FA012802D09C
:108120000BA0FAF735FA1CBD44020020FD810008BF
:10813000DC3700208581000869810008E1810008A2
:10814000503800207368656C6C000000B97A000834
:108150007368656C6C207461736B20637265617405
:10816000206661696C65640010B5044600235A1EE0
:1081700019460348006800F0F5FE002010BD00001D
:108180004402002070B504460D4600F005F81420A6
:1081900000F0DCFA002070BD10B50D480078A8B1E1
:1081A000002406E00B48015D0B48FEF717FE601C3B
:1081B000C4B20A4800888442F4DD002007490880E0
:1081C00003490870FF210348F8F713F810BD0000B9
:1081D00058000020B4040020DC3700205A000020A2
:1081E00010B5044600231A4619460348006800F0FB
:1081F000FDFF002010BD00004402002070B50446C1
:108200000D4621460248FAF778F928B270BD000001
:108210000038014038B54FF4A8715448F7F7E9FF2A
:108220005348524908615348486153494F48C16215
:1082300052490163524981645249C16452494166BD
:10824000524981665249C0F880105249C0F88410E2
:108250005149C0F89C105149C0F8A0105049C0F8CD
:10826000B8105049C0F8BC104F49C0F8D4104F495D
:10827000C0F8D8104E49C0F8F0104E49C0F8F410BC
:108280004D49C0F80C114D49C0F810114C49C0F8C7
:1082900028114C49C0F82C114B49C0F844114B49E6
:1082A000C0F8481101210D20F9F7F2FC01214848DE
:1082B000F9F70EFA4FF2E220ADF8000048208DF8F1
:1082C000030069464348F9F778F941F60100ADF833
:1082D000000028208DF8030069463F48F9F76DF942
:1082E0002248007820F00100401C2049087014202A
:1082F000088150204881C82088814FF49670C88139
:108300000846FCF767FA01242CE0C4EBC4001749C7
:1083100011F8200020F00100C4EBC401134A02F858
:1083200021001420C4EBC40102EB8101088150201C
:10833000C4EBC40102EB81014881C820C4EBC40135
:1083400002EB810188814FF49670C4EBC40102EB0B
:108350008101C881C4EBC40102EB8100FCF73AFA49
:10836000601CC4B20C2CD0DB38BD000064030020BC
:108370005D340008853100086D34000801320008C2
:10838000813400084532000895340008893200081D
:10839000A5340008CD320008B934000811330008B4
:1083A000C934000855330008DD340008993300084B
:1083B000ED340008DD33000829340008753000086A
:1083C00039340008C130000849340008553100082C
:1083D00000023000000C01400008014001460A691B
:1083E000D1E901309860D1E90103586050688842B2
:1083F00001D188685060002008611068401E10603C
:108400001068704700F1080141604FF0FF31816052
:1084100000F10801C1600161002101607047002185
:108420000161704710B502460B685C1C0CB91069FD
:1084300007E002F1080000E04068446824689C42BC
:10844000FAD944684C604C68A160886041600A6158
:108450001468641C146010BD42684A6093688B60A5
:10846000936859609160086103685B1C0360704702
:1084700010B500BF502080F31188BFF34F8FBFF3BA
:108480006F8F00BF0B480068401C0A49086008460F
:10849000006801280DD108480068C0B208B9012061
:1084A00000E0002028B94FF4BD7204A10DA0FAF736
:1084B0006FF810BDA401002004ED00E02E2E5C2E0C
:1084C0002E5C4672656552544F535C706F72745CDB
:1084D000525644535C41524D5F434D335C706F7252
:1084E000742E63004572726F723A25732C25640DE9
:1084F0000A00000010B50B48006828B940F281124C
:1085000009A113A0FAF744F806480068401E05497F
:1085100008600846006820B9002080F3118800BF79
:1085200000BF10BDA40100202E2E5C2E2E5C4672D2
:10853000656552544F535C706F72745C525644536D
:108540005C41524D5F434D335C706F72742E63001B
:108550004572726F723A25732C25640D0A00000073
:1085600070B506463546002E35D0083D2C461A49D2
:1085700060680968084008B1012000E0002028B9BF
:108580004FF4A07215A11FA0FAF702F8206808B9ED
:10859000012000E0002028B940F241120FA119A0EB
:1085A000F9F7F6FF0C4960680968084098B120683F
:1085B00088B90949606809688843606000F0D0FAAA
:1085C0001449606809680844124908602046FDF7AC
:1085D000F9F901F081F970BDA00100202E2E5C2E6A
:1085E0002E5C4672656552544F535C706F72745CBA
:1085F0004D656D4D616E675C686561705F342E63BB
:10860000000000004572726F723A25732C25640DCC
:108610000A00000098010020064800684FF47A71B3
:10862000B0FBF1F0401E4FF0E021486107200861E7
:1086300070470000C401002070B5F7F7ABFD054698
:10864000102D11D305F1E02090F8F0431048007888
:10865000844201DB012000E0002028B94FF42A7297
:108660000CA116A0F9F794FF1848006800F4E06028
:1086700017490968884201D8012000E0002028B984
:108680004FF42E7203A10DA0F9F782FF70BD000018
:10869000A80100202E2E5C2E2E5C46726565525479
:1086A0004F535C706F72745C525644535C41524D30
:1086B0005F434D335C706F72742E63004572726F4E
:1086C000723A25732C25640D0A0000000CED00E0C1
:1086D000AC010020024600200BE0084B53F830307C
:1086E00033B9064B43F8301003EBC0035A6002E085
:1086F000401C0A28F1D300BF70470000580A002030
:108700002DE9F04105460E4617462C46FFF7B0FE10
:1087100094F94400401C10B9002084F8440094F9F6
:108720004500401C10B9002084F84500FFF7E2FE28
:10873000A06B28B93A46314604F1240000F002F952
:108740002046FDF792FBBDE8F081000070B50446BD
:108750000025ACB10F48006808B9012000E00020F6
:1087600028B940F2CF420CA112A0F9F711FF00F096
:10877000F7F900212046FCF765FE01F0ADF805464B
:108780003DB94FF080500F490860BFF34F8FBFF3E2
:108790006F8F70BD740100202E2E5C2E2E5C4672F1
:1087A000656552544F535C7372635C7461736B7391
:1087B0002E6300004572726F723A25732C25640D8A
:1087C0000A00000004ED00E070B50546FFF750FE1A
:1087D00015B92D48006800E028460446201DFFF723
:1087E000FDFD78B9E06A00EB8000284951F82000CF
:1087F00040B994F82C10012088402549096881432C
:1088000023480160A06A18B104F11800FFF7E6FDE3
:1088100020480068401C1F4908601B4800688442CB
:1088200009D1211D1C48FFF717FE1C480068401C99
:108830001A49086009E01A480068401E1849086093
:108840002046FCF75CFFFDF73DFAFFF753FE1548A5
:108850000068C0B10C480068844214D11248006816
:1088600008B9012000E0002028B940F265420FA1BC
:1088700015A0F9F78DFE4FF0805017490860BFF33F
:108880004F8FBFF36F8F70BD3C010020A80A0020FE
:108890005401002068010020640D002048010020E0
:1088A0004C01002058010020740100202E2E5C2E67
:1088B0002E5C4672656552544F535C7372635C74F0
:1088C00061736B732E6300004572726F723A257389
:1088D0002C25640D0A00000004ED00E00120014990
:1088E000086070476001002070B504460D462CB941
:1088F00040F6063207A10EA0F9F74AFE10480168BB
:1089000018312046FFF78EFD01212846FCF79AFD1D
:1089100070BD00002E2E5C2E2E5C46726565525492
:108920004F535C7372635C7461736B732E630000EE
:108930004572726F723A25732C25640D0A0000008F
:108940003C01002070B505460E4614462DB940F690
:10895000313209A10FA0F9F71BFE12480168183146
:108960002846FFF779FD0CB14FF0FF36214630461F
:10897000FCF768FD70BD00002E2E5C2E2E5C46724A
:10898000656552544F535C7372635C7461736B73AF
:108990002E6300004572726F723A25732C25640DA8
:1089A0000A0000003C01002070B505462C46002D51
:1089B0004BD02649E06A0968C96A884245D2A06955
:1089C00000F0004028B921480068C06AC0F12000CA
:1089D000A061E16A01EB81011D4A02EB810160693E
:1089E000884201D1012000E0002050B3201DFFF794
:1089F000F5FC78B9E06A00EB8000154951F82000D9
:108A000040B994F82C10012088401249096881432C
:108A1000104801600D480068C06AE06294F82C10AC
:108A2000012088400B49096808430A490860E16A47
:108A300001EB8101064A02EB8100211DFFF70CFDCD
:108A400003E002480068C06AE06270BD3C0100209B
:108A5000A80A00205401002010B504462CB940F6A5
:108A6000C13205A10BA0F9F793FD0E480068206004
:108A70000D480068606010BD2E2E5C2E2E5C467284
:108A8000656552544F535C7372635C7461736B73AE
:108A90002E6300004572726F723A25732C25640DA7
:108AA0000A00000064010020500100201CB51A4893
:108AB00000210B468022CDE9001018A1194800F0D2
:108AC00043FD0446012C02D100F0B2FF0446012C04
:108AD00015D100BF502080F31188BFF34F8FBFF333
:108AE0006F8F00BF4FF0FF300F49086001200F4922
:108AF000086000200E49086000F07AF90BE0601C65
:108B000008B1012000E0002028B940F2847209A1D8
:108B10000FA0F9F73DFD1CBD7001002049444C45F4
:108B200000000000B55700086C010020580100202B
:108B3000500100202E2E5C2E2E5C4672656552542C
:108B40004F535C7372635C7461736B732E630000CC
:108B50004572726F723A25732C25640D0A0000006D
:108B600002480068401C01490860704774010020F9
:108B700010B51B48006818B101201A4908602DE0A3
:108B800000201849086018480068B0FA80F0C0F169
:108B90001F0404EB8400154951F8200008B101209E
:108BA00000E0002028B940F6F62211A117A0F9F73D
:108BB000EFFC04EB84010D4A02EB81004168496837
:108BC000416000F1080142688A4202D14168496867
:108BD00041604168C968114A116000BF10BD0000C2
:108BE000740100206001002054010020A80A002028
:108BF0002E2E5C2E2E5C4672656552544F535C736C
:108C000072635C7461736B732E6300004572726FE4
:108C1000723A25732C25640D0A0000003C010020E7
:108C20003EB50446FEF794F80546002000900190FA
:108C30000290002D2AD0012C28DB072C26DC2246AE
:108C400014A16846F9F7CEFC4FF480711448F8F788
:108C500092FD144807226946C3681348984741F2B9
:108C60008830FFF773FD0F4807226946C3680E4836
:108C7000984740F6C410FFF769FD4FF4807108482B
:108C8000F8F777FD09A0F9F783FC02E00DA0F9F7EA
:108C90007FFC3EBD6C6576656C302564000000008D
:108CA000000C01404400002000440040E99FB3E96B
:108CB000878FE8AEBEE7BDAEE68890E58A9F200AC2
:108CC00000000000E8BE93E585A5E697A0E695883C
:108CD0002CE99FB3E9878FE88C83E59BB420312D85
:108CE00037200A0070B506460C46002501230622EF
:108CF0002146304600F00EF805460DB1284670BDFD
:108D0000142204F1140106F11400FBF77BFA054666
:108D10002846F4E72DE9F84380460D4616461F46DF
:108D20004FF00009B7420AD3154816A31CA24FF40E
:108D30008871009022A0FBF791F900BFFEE755B9BA
:108D40000F4827A316A240F2111100901CA0FBF7B8
:108D500085F900BFFEE73A4631462846FDF76AFC32
:108D60000446601C10B90020BDE8F883291908EBFF
:108D700004000422FBF746FA81464846F4E7000067
:108D80004C9B00087374617475735F696E646578D9
:108D9000203C207374617475735F6E756D00000004
:108DA00028257329206861732061737365727420AC
:108DB0006661696C65642061742025732E0A000069
:108DC0002E2E5C2E2E5C557365725C656173796422
:108DD000625C7372635C65665F656E762E6300002D
:108DE0007374617475735F7461626C650000000078
:108DF0001CB52248014609780191FF2102461170F5
:108E00000146097800919DF8001001F050011C4ABC
:108E1000117007211B4A116009E01A490968491EAF
:108E2000184A11609DF800104906090E00919DF83E
:108E3000001001F080018029EFD012490968090271
:108E4000104A11601146098801F4E06111600B4A73
:108E5000019911700C48006840F470000A490860DC
:108E60000846006840F070400860FFF7D5FB00201E
:108E700006490860F7F758F900201CBD00E400E03F
:108E8000A8010020AC01002020ED00E0A40100209A
:108E900010B500BF502080F31188BFF34F8FBFF390
:108EA0006F8F00BF00F096FB18B14FF0805004495F
:108EB000086000BF002080F3118800BF10BD0000D3
:108EC00004ED00E02DE9F04104460126002722468A
:108ED0000021012000F008F805462846FCF77EFC3A
:108EE0002846BDE8F08100002DE9F84305460E460E
:108EF00090460DB1012000E0002028B94FF4C47263
:108F00000DA114A0F9F744FB0EB9002701E005FB01
:108F100006F707F14800FCF7E7FF044644B104F107
:108F2000480943464A46314628460094FCF764FC0B
:108F30002046BDE8F88300002E2E5C2E2E5C467283
:108F4000656552544F535C7372635C7175657565EA
:108F50002E6300004572726F723A25732C25640DE2
:108F60000A0000002DE9FF4782B005460E461F4665
:108F70004FF0000A2C462CB940F2DC4261A168A0F7
:108F8000F9F706FB0EB9206C08B9012000E00020BB
:108F900028B940F2DD425BA161A0F9F7F9FA00F0CF
:108FA00003FB08B9049808B9012000E0002028B9A3
:108FB0004FF49C6253A15AA0F9F7EAFA00BFFFF7F9
:108FC00057FAD4F83890B9F1000F3DD0D4F80C809E
:108FD00031462046FCF740FBDFB9A9F10100A06350
:108FE000206810B9FDF72AF86060206908B90120EF
:108FF00000E0002010BB04F1100000F00FFCE8B10D
:109000004FF080504A490860BFF34F8FBFF36F8F16
:1090100014E0C4F80C80606A08B9012000E0002068
:1090200060B904F1240000F0F9FB38B14FF0805032
:109030003F490860BFF34F8FBFF36F8FFFF75AFAB6
:10904000012006B0BDE8F087049818B9FFF752FA7E
:109050000020F6E7BAF1000F04D16846FFF7FCFCE8
:109060004FF0010AFFF746FAFFF77AFDFFF700FA23
:1090700094F94400401C10B9002084F8440094F98D
:109080004500401C10B9002084F84500FFF732FA73
:1090900004A9684600F004FA40BB2046FCF7F2FC45
:1090A000F0B1206830B9FFF7E3F96068FFF77CFCA6
:1090B000FFF720FA04F124000499FFF715FC20467D
:1090C000FCF7D3FE00F008FC00287FF478AF4FF0E7
:1090D000805017490860BFF34F8FBFF36F8F6EE763
:1090E0002046FCF7C2FE00F0F7FB68E72046FCF7DD
:1090F000BCFE00F0F1FB2046FCF7C4FC0028EED0DB
:1091000000209EE72E2E5C2E2E5C46726565525422
:109110004F535C7372635C71756575652E630000F7
:109120004572726F723A25732C25640D0A00000097
:1091300004ED00E070B505460E462C462CB940F211
:109140001B121EA124A0F9F723FAFFF791F9D4E925
:109150000F12206801FB020060600020A0632068FD
:10916000A060E06B401E226C216800FB0210E060F2
:10917000FF2084F8440084F845009EB9206908B9AE
:10918000012000E00020A8B904F1100000F046FB27
:1091900080B14FF0805014490860BFF34F8FBFF388
:1091A0006F8F07E004F11000FFF72CF904F12400A1
:1091B000FFF728F9FFF79EF9012070BD2E2E5C2ED7
:1091C0002E5C4672656552544F535C7372635C71DA
:1091D000756575652E6300004572726F723A25736E
:1091E0002C25640D0A00000004ED00E02DE9FF438A
:1091F00083B0064688461D464FF0000934462CB918
:1092000040F2D92258A15FA0F9F7C2F9B8F1000FD6
:1092100001D1206C08B9012000E0002028B940F2FB
:10922000DA2251A157A0F9F7B3F9022D02D1E06B70
:10923000012801D1012000E0002028B940F2DB2202
:1092400049A150A0F9F7A4F900F0AEF908B90598C2
:1092500008B9012000E0002028B940F2DE2242A136
:1092600048A0F9F795F900BFFFF702F9A06BE16B91
:10927000884201D3022D28D12A4641462046FCF7D8
:1092800000FA0746606A08B9012000E0002068B9CA
:1092900004F1240000F0C2FA88B14FF080503D493B
:1092A0000860BFF34F8FBFF36F8F08E03FB14FF0FF
:1092B000805038490860BFF34F8FBFF36F8FFFF7BF
:1092C00019F9012007B0BDE8F083059818B9FFF738
:1092D00011F90020F6E7B9F1000F04D101A8FFF75A
:1092E000BBFB4FF00109FFF705F9FFF739FCFFF76A
:1092F000BFF894F94400401C10B9002084F84400E1
:1093000094F94500401C10B9002084F84500FFF78F
:10931000F1F805A901A800F0C3F8F0B92046FCF760
:10932000BEFBA0B104F110000599FFF7DDFA20465D
:10933000FCF79BFD00F0D0FA002895D14FF080504B
:1093400014490860BFF34F8FBFF36F8F8CE720463F
:10935000FCF78BFD00F0C0FA86E72046FCF785FDA0
:1093600000F0BAFA0020ADE72E2E5C2E2E5C46727D
:10937000656552544F535C7372635C7175657565B6
:109380002E6300004572726F723A25732C25640DAE
:109390000A00000004ED00E02DE9F05F07468A4670
:1093A00090461E463C462CB940F29F3231A138A06F
:1093B000F9F7EEF8BAF1000F01D1206C08B90120DD
:1093C00000E0002028B94FF468722AA130A0F9F714
:1093D000DFF8022E02D1E06B012801D1012000E06C
:1093E000002028B940F2A13222A129A0F9F7D0F833
:1093F000FFF722F900BF5021EFF3118081F31188AC
:10940000BFF34F8FBFF36F8F00BF0546A06BE16BBB
:10941000884201D3022E23D194F945B032465146F9
:109420002046FCF72EF90BF1010088B9606A08B9F3
:10943000012000E0002080B904F1240000F0EEF9E2
:1094400058B1B8F1000F08D00120C8F8000004E0BE
:109450000BF1010040B284F845004FF0010901E032
:109460004FF0000900BF85F3118800BF4846BDE8F2
:10947000F09F00002E2E5C2E2E5C467265655254C5
:109480004F535C7372635C71756575652E63000084
:109490004572726F723A25732C25640D0A00000024
:1094A0002DE9F04104460D462CB940F6CB3219A106
:1094B0001FA0F9F76DF82DB940F6CC3215A11CA00C
:1094C000F9F766F8FEF7D4FF1D4807682868401CC6
:1094D00008B9002619E01B4920680968884204D0B1
:1094E0006068B84201D801260FE06068381A296820
:1094F000884209D228686168791A401A2860204693
:10950000FFF7AAFA002600E00126FEF7F3FF304637
:10951000BDE8F0812E2E5C2E2E5C4672656552549D
:109520004F535C7372635C7461736B732E630000E2
:109530004572726F723A25732C25640D0A00000083
:1095400050010020640100202DE9FF4F85B08046C6
:1095500089461746DDE912ABB800FCF7C5FC0646A4
:1095600056B15420FCF7C0FC04460CB1266304E05D
:109570003046FEF7F5FF00E000247CB10020CDE985
:1095800000ABCDE902403A4649464046089BFCF70D
:1095900047F92046FBF7A2FF012501E04FF0FF3518
:1095A000284609B0BDE8F08F0549096809B90120CE
:1095B00005E00449096809B9022000E0002070476D
:1095C000580100207401002001490868704700001C
:1095D000500100202DE9F0414FF00008414800689B
:1095E000002872D140480068451C3F480560EDB92D
:1095F0003E480068006808B9012000E0002028B952
:1096000040F6D9123AA141A0F8F7C2FF37480768DF
:109610004248006835490860404807604048006893
:10962000401C3F490860FCF74DFB00BF3D48006807
:1096300085423CD300BF2D480068006808B901206E
:1096400000E0002020B14FF0FF30364908602DE0E7
:1096500026480068C068C4686668B54202D23148CE
:10966000066023E0201DFEF7B9FEA06A18B104F1E0
:109670001800FEF7B3FE94F82C10012088402A4908
:109680000968084328490860E16A01EB8101274A1B
:1096900002EB8100211DFEF7DFFE2549E06A096823
:1096A000C96A8842C7D34FF00108C4E700BF204809
:1096B0000068C06A00EB80001C4951F820000128B6
:1096C00001D94FF0010805E0FFE71A480068401C87
:1096D000184908601848006808B14FF00108404672
:1096E000BDE8F081740100205001002040010020FD
:1096F0002E2E5C2E2E5C4672656552544F535C7361
:1097000072635C7461736B732E6300004572726FD9
:10971000723A25732C25640D0A00000044010020D4
:10972000640100206C01002054010020A80A0020E0
:109730003C0100205C0100206001002070B505465E
:109740002C460026002D4BD026480068844201D1CB
:10975000012000E0002028B940F6C76222A129A01C
:10976000F8F716FFA06C28B940F6C9621EA125A023
:10977000F8F70EFFA06C401EA064616CE06A88429E
:109780002ED0A06C60BB201DFEF728FE78B9E06AE1
:1097900000EB80001F4951F8200040B994F82C10CC
:1097A000012088401C49096881431B480160606CA6
:1097B000E062E06AC0F12000A06194F82C10012062
:1097C000884015490968084313490860E16A01EBBC
:1097D0008101104A02EB8100211DFEF73DFE0126AA
:1097E000304670BD3C0100202E2E5C2E2E5C467251
:1097F000656552544F535C7372635C7461736B7331
:109800002E6300004572726F723A25732C25640D29
:109810000A000000A80A00205401002070B5064686
:10982000F068C4682CB940F661321AA120A0F8F79C
:10983000AFFE04F11800FEF7D1FD21480068A8B979
:10984000201DFEF7CBFD94F82C10012088401D4907
:10985000096808431B490860E16A01EB81011A4A63
:1098600002EB8100211DFEF7F7FD04E004F1180171
:109870001648FEF7F1FD1649E06A0968C96A884290
:1098800004D9012501201349086000E0002528467D
:1098900070BD00002E2E5C2E2E5C46726565525403
:1098A0004F535C7372635C7461736B732E6300005F
:1098B0004572726F723A25732C25640D0A00000000
:1098C0007401002054010020A80A0020500D00203F
:1098D0003C0100206001002070B5002400263448BF
:1098E000006828B94FF4FD6232A139A0F8F750FEA4
:1098F000FEF7BEFD2E480068401E2D490860084650
:10990000006800284FD13648006800284BD024E07A
:109910003448C068C46804F11800FEF75FFD201DDC
:10992000FEF75CFD94F82C10012088402E49096850
:1099300008432D490860E16A01EB81012B4A02EBE3
:109940008100211DFEF788FD2949E06A0968C96A7E
:10995000884202D30120274908602248006808B9DC
:10996000012000E000200028D2D00CB1FCF7AAF9B9
:109970002148056865B100BFFFF72CFE10B101203A
:109980001C4908606D1E002DF6D100201A490860A0
:109990001848006838B10126300718490860BFF33D
:1099A0004F8FBFF36F8FFEF7A5FD304670BD0000EF
:1099B000740100202E2E5C2E2E5C4672656552547A
:1099C0004F535C7372635C7461736B732E6300003E
:1099D0004572726F723A25732C25640D0A000000DF
:1099E0004C010020500D002054010020A80A002046
:1099F0003C010020600100205C01002004ED00E03B
:109A00002DE9FC4705460E4617469846DDF8289096
:109A10002820FCF769FA04463CB143463A463146F1
:109A20002846CDE90094FBF761FF2046BDE8FC879E
:109A30001CB50024FBF7ACFD0B48006850B10B4887
:109A40001F2100238022CDE9001009A10A48FFF759
:109A50007BFD04462CB940F2331208A10EA0F8F7A2
:109A600097FD20461CBD00008001002084010020DD
:109A7000546D722053766300515E00082E2E5C2ECA
:109A80002E5C4672656552544F535C7372635C740E
:109A9000696D6572732E63004572726F723A257339
:109AA0002C25640D0A0000002DE9FE4304460D46F6
:109AB00016461F46DDF828804FF000092CB94FF4F8
:109AC000D37216A11CA0F8F763FD1F48006810B3FD
:109AD000009501960294062D15DAFFF765FD022820
:109AE00008D100234246694617480068FFF77EFB0D
:109AF000814610E000231A46694613480068FFF7C4
:109B000075FB814607E000233A4669460E48006827
:109B1000FFF742FC81464846BDE8FE832E2E5C2EB0
:109B20002E5C4672656552544F535C7372635C746D
:109B3000696D6572732E63004572726F723A257398
:109B40002C25640D0A0000008001002077726974E2
:109B5000655F73746174757300726561645F7374BB
:109B60006174757300726561645F656E760072651D
:109B700061645F736563746F725F6D6574615F6468
:109B80006174610065665F726561645F656E765FD2
:109B900076616C756500666F726D61745F73656385
:109BA000746F720065665F656E765F7365745F647F
:109BB000656661756C740065665F656E765F696E7B
:109BC0006974000000000000963007772C610EEEEB
:109BD000BA51099919C46D078FF46A7035A563E904
:109BE000A395649E3288DB0EA4B8DC791EE9D5E02B
:109BF00088D9D2972B4CB609BD7CB17E072DB8E72A
:109C0000911DBF906410B71DF220B06A4871B9F37E
:109C1000DE41BE847DD4DA1AEBE4DD6D51B5D4F4B7
:109C2000C785D38356986C13C0A86B647AF962FD1C
:109C3000ECC9658A4F5C0114D96C0663633D0FFA69
:109C4000F50D088DC8206E3B5E10694CE44160D56F
:109C5000727167A2D1E4033C47D4044BFD850DD259
:109C60006BB50AA5FAA8B5356C98B242D6C9BBDB6C
:109C700040F9BCACE36CD832755CDF45CF0DD6DC67
:109C8000593DD1ABAC30D9263A00DE518051D7C80E
:109C90001661D0BFB5F4B42123C4B3569995BACF99
:109CA0000FA5BDB89EB802280888055FB2D90CC6BA
:109CB00024E90BB1877C6F2F114C6858AB1D61C133
:109CC0003D2D66B69041DC760671DB01BC20D29852
:109CD0002A10D5EF8985B1711FB5B606A5E4BF9FDF
:109CE00033D4B8E8A2C9077834F9000F8EA80996D2
:109CF00018980EE1BB0D6A7F2D3D6D08976C64913D
:109D0000015C63E6F4516B6B62616C1CD830658555
:109D10004E0062F2ED95066C7BA5011BC1F4088232
:109D200057C40FF5C6D9B06550E9B712EAB8BE8B73
:109D30007C88B9FCDF1DDD62492DDA15F37CD38CFC
:109D4000654CD4FB5861B24DCE51B53A7400BCA3FA
:109D5000E230BBD441A5DF4AD795D83D6DC4D1A42C
:109D6000FBF4D6D36AE96943FCD96E34468867AD03
:109D7000D0B860DA732D0444E51D03335F4C0AAAA2
:109D8000C97C0DDD3C710550AA41022710100BBEA5
:109D900086200CC925B56857B3856F2009D466B9EC
:109DA0009FE461CE0EF9DE5E98C9D9292298D0B021
:109DB000B4A8D7C7173DB359810DB42E3B5CBDB7CE
:109DC000AD6CBAC02083B8EDB6B3BF9A0CE2B6034F
:109DD0009AD2B1743947D5EAAF77D29D1526DB0404
:109DE0008316DC73120B63E3843B64943E6A6D0D4F
:109DF000A85A6A7A0BCF0EE49DFF099327AE000A9A
:109E0000B19E077D44930FF0D2A3088768F2011E2C
:109E1000FEC206695D5762F7CB67658071366C19C3
:109E2000E7066B6E761BD4FEE02BD3895A7ADA10E4
:109E3000CC4ADD676FDFB9F9F9EFBE8E43BEB717C5
:109E4000D58EB060E8A3D6D67E93D1A1C4C2D8384F
:109E500052F2DF4FF167BBD16757BCA6DD06B53FB5
:109E60004B36B248DA2B0DD84C1B0AAFF64A0336F4
:109E7000607A0441C3EF60DF55DF67A8EF8E6E3173
:109E800079BE69468CB361CB1A8366BCA0D26F25BC
:109E900036E2685295770CCC03470BBBB916022209
:109EA0002F260555BE3BBAC5280BBDB2925AB42B1E
:109EB000046AB35CA7FFD7C231CFD0B58B9ED92C33
:109EC0001DAEDE5BB0C2649B26F263EC9CA36A7598
:109ED0000A936D02A906099C3F360EEB856707724F
:109EE00013570005824ABF95147AB8E2AE2BB17BB6
:109EF000381BB60C9B8ED2920DBED5E5B7EFDC7C3D
:109F000021DFDB0BD4D2D38642E2D4F1F8B3DD6893
:109F10006E83DA1FCD16BE815B26B9F6E177B06F8E
:109F20007747B718E65A0888706A0FFFCA3B06667B
:109F30005C0B0111FF9E658F69AE62F8D3FF6B6108
:109F400045CF6C1678E20AA0EED20DD75483044EAA
:109F5000C2B30339612667A7F71660D04D47694938
:109F6000DB776E3E4A6AD1AEDC5AD6D9660BDF404B
:109F7000F03BD83753AEBCA9C59EBBDE7FCFB247FE
:109F8000E9FFB5301CF2BDBD8AC2BACA3093B353E3
:109F9000A6A3B4240536D0BA9306D7CD2957DE54EC
:109FA000BF67D9232E7A66B3B84A61C4021B685DC5
:109FB000942B6F2A37BE0BB4A18E0CC31BDF055A3E
:109FC0008DEF022D40A30008F4A10008000000005E
:109FD00065665F706F72745F6572617365007A6940
:109FE0006974005A494954313233340064656661FA
:109FF000756C7420757365720073657456617200B8
:10A000007365742076617200757000646F776E00FE
:10A010007269676874006C656674007461620062DE
:10A0200061636B7370616365006261636B73706120
:10A0300063650064656C65746500656E74657200C7
:10A040007573657273006C69737420616C6C207534
:10A0500073657200726F6F740061646D696E007277
:10A060006F6F74207573657200636D6473006C6943
:10A07000737420616C6C20636D6400766172730090
:10A080006C69737420616C6C2076617200636C651E
:10A09000617200636C65617220636F6E736F6C65D3
:10A0A000004154004C6F7261E9808FE4BCA0006BEA
:10A0B00065795F7300E8AEBEE7BDAEE99481E5AEB9
:10A0C0009AE697B6E997B42033202D2032307300FA
:10A0D0006B65795F656E5F7265616400E69FA5E8F8
:10A0E000AFA2E68C89E994AEE4BDBFE883BD006B06
:10A0F00065795F656E5F73657400E8AEBEE7BDAEFF
:10A10000E68C89E994AEE4BDBFE883BD00766F6C50
:10A110005F73657400E4BFAEE694B9E8AEBEE5A433
:10A1200087E99FB3E9878F20696E73203A20312039
:10A130002D2037007379735F696E697400E5889D1F
:10A14000E5A78BE58C96E7B3BBE7BB9FE58F82E67F
:10A1500095B028E585A8E68C89E994AEE4BDBFE812
:10A1600083BD2C20313073E4BC91E79CA029000012
:10A1700040404040404040404041414141414040DA
:10A1800040404040404040404040404040404040CF
:10A19000050202020202020202020202020202029C
:10A1A0002020202020202020202002020202020263
:10A1B00002909090909090101010101010101010AD
:10A1C00010101010101010101010100202020202D5
:10A1D0000288888888888808080808080808080805
:10A1E00008080808080808080808080202020240CF
:10A1F00070A10008300000003100000033000000B2
:10A200003400000035000000360000003700000078
:10A210005761726E696E673A20536563746F72207E
:10A2200068656164657220636865636B2066616957
:10A230006C65642E20466F726D617420746869735A
:10A2400020736563746F7220283078253038782940
:10A250002E0A0000466F756E6420616E20454E56D2
:10A260002028252E2A732920776869636820686171
:10A2700073206368616E6765642076616C75652024
:10A280006661696C65642E204E6F772077696C6C0F
:10A29000207265636F766572792069742E0A0000FA
:10A2A0005761726E696E673A20416C6C6F63206112
:10A2B0006E20454E56202873697A65202564292032
:10A2C0006661696C6564207768656E206E657720CD
:10A2D000454E562E204E6F772077696C6C20474391
:10A2E000207468656E2072657472792E0A00000011
:10A2F0005761726E696E673A204D6F7665642061B2
:10A300006E20454E56202873697A652025642920E1
:10A310006661696C6564207768656E207265636F3D
:10A32000766572792E204E6F772077696C6C2047A6
:10A3300043207468656E2072657472792E0A00007D
:10A34000626F6F745F74696D657300000D0A436F0F
:10A350006D6D616E64204C6973743A0D0A000000E3
:10A360000D0A566172204C6973743A0D0A000000A0
:10A370000D0A55736572204C6973743A0D0A00001A
:10A380000D0A4B6579204C6973743A0D0A00000080
:10A39000436F6D6D616E64206E6F7420466F756ED5
:10A3A000640D0A000D0A5761726E696E673A2043A8
:10A3B0006F6D6D616E6420697320746F6F206C6FB8
:10A3C0006E670D0A00000000206973206E6F742014
:10A3D00061207661720D0A0063616E2774207365D7
:10A3E000742072656164206F6E6C79207661720DE5
:10A3F0000A00000063616E27742073657420706F1B
:10A40000696E7465720D0A000D0A70617373776F5F
:10A410007264206572726F720D0A000056617220BC
:10A420006E6F7420466F756E740D0A000D0A383811
:10A43000383838383838383850203838383838389C
:10A4400038203838383838383820383838383838BC
:10A450003838383838200D0A202020202020643851
:10A46000385020202020383838202020202038382C
:10A47000382020202020202038383820202020207C
:10A480000D0A202020202064383850202020202051
:10A49000383838202020202038383820202020202C
:10A4A000202038383820202020200D0A202020208D
:10A4B00064383850202020202020383838202020B0
:10A4C00020203838382020202020202038383820FC
:10A4D000202020200D0A2020206438385020202001
:10A4E00020202020383838202020202038383820DC
:10A4F00020202020202038383820202020200D0A3D
:10A500002020643838502020202020202020383877
:10A5100038202020202038383820202020202020DB
:10A5200038383820202020200D0A20643838502068
:10A5300020202020202020203838382020202020D3
:10A54000383838202020202020203838382020207B
:10A5500020200D0A643838383838383838383820F0
:10A56000383838383838382038383838383838209B
:10A570002020202038383820202020200D0A0D0AE5
:10A580004275696C643A202020202020204D6172A1
:10A5900020333120323032362030393A30323A35B9
:10A5A000300D0A56657273696F6E3A2020202020A4
:10A5B000332E322E340D0A436F70797269676874D6
:10A5C0003A202020286329203230323520E4B8ADEB
:10A5D000E5B7A5E5889BE699BA0D0A001B5B324BEF
:10A5E0000D0000002020434D442000005641522021
:10A5F000000000004B45592000000000636F6D6DA6
:10A60000616E642068656C70206F66200000000039
:10A61000506C6561736520696E707574207061732C
:10A6200073776F72643A00004E4F4E450000000091
:10A630001B5B324A1B5B31480000000055534552FA
:10A6400000000000C4A70008000000205002000025
:10A65000260B0008A4A8000850020020003B0000C0
:10A660004826000800080000DE9F0008E39F00085D
:10A67000EC9F000800210000F99F000829760008DF
:10A6800000A000080009000000415B1B6B7B000874
:10A6900008A000080009000000425B1B7D6800085C
:10A6A0000BA000080019000000435B1B8374000826
:10A6B00010A000080019000000445B1BED710008A9
:10A6C00016A0000800090000000000093579000804
:10A6D0001BA0000800190000000000088D6600089B
:10A6E0001FA00008001900000000007F8D66000810
:10A6F00029A00008001900007E335B1B7367000867
:10A7000033A00008001900000000000D8D6800084B
:10A710003AA000080021000040A00008797B000852
:10A7200046A00008FF08000054A0000859A0000837
:10A730005FA000080021000069A000086167000810
:10A740006EA00008002100007BA000088B7B0008A1
:10A7500080A00008002100008DA000081D670008EF
:10A7600093A0000800210100A1A00008A151000849
:10A77000A4A0000800210100AFA00008C911000832
:10A78000B5A0000800210000D0A00008994E0008E4
:10A79000DCA0000800210000EFA000084D500008D8
:10A7A000FAA00008002100000DA10008218C00087B
:10A7B00015A100080021000034A100082D7D00082B
:10A7C0003DA10008011813F90F14083510420813B1
:10A7D0007D0B1408214A1408F51714084D181B089E
:10A7E0007D0813851D14085D121C0855250C121FC9
:10A7F0001408A5201408D92114086F241B08A104EB
:10A8000001181AFF014113DD7E140808A21408F88C
:10A81000A15B08F4041AFC04A910DA0C20DA041075
:10A8200011D9102950690C6950A9102950A9102973
:10A8300050A9102950A9106904A964A91401681A23
:10A84000AA01C12D01020304041808060708090221
:10A850000406B8AB4A041C29180114132CA41408CC
:10A86000A4A31B084C041A60041A70041A80041A6A
:10A8700090041AF4041AD8041AC8041A1C2813FCE9
:10A88000A5140810A61B08080C1A30081ADC101AA8
:10A89000E4041AEC041A3C101AF4081A2808E322FB
:04A8A0002200000092
:04000005080000ED02
:00000001FF
